:020000040800F2
:10400000005000204D74000821730008257300083B
:10401000297300082D7300083173000800000000A8
:1040200000000000000000000000000039730008DC
:1040300035730008000000003D73000899970008E0
:104040004173000845730008497300084D73000868
:104050005173000855730008597300085D73000818
:104060000000000061730008657300080000000094
:104070000000000000000000000000000000000040
:10408000000000000000000085730008897300082C
:1040900099730008A9730008C573000869450008F2
:1040A000D5730008CD4900080000000000000000A2
:1040B00055460008A545000829460008D9730008A0
:1040C000DD730008E1730008E5730008E973000878
:1040D000ED730008F1730008F5730008ED44000863
:1040E000FD7300080174000805740008000000005A
:1040F00000000000000000000000000000000000C0
:0C41000000000000000000005FF800005C
:10410C0030BF704720BF704740BF7047BFF36F8F01
:10411C007047BFF34F8F7047BFF35F8F704701DF5E
:10412C007047EFF31480704780F31488BFF36F8FE0
:10413C007047EFF30980704780F309887047EFF3FD
:10414C000880704780F30888704772B6704762B673
:10415C00704771B6704761B6704780F3118870472D
:10416C00EFF31280704740BA704700BA70470000F6
:10417C00054A0649064B1160064A1360064A13604D
:10418C00064A1360704700BF800400202587000892
:10419C00DD8500085C04002024030020540400206A
:1041AC00064A074B1A60074A074B1A60074A084B26
:1041BC001A60084A084B1A60704700BF9DA6000899
:1041CC0024030020A9A80008800400209DA8000852
:1041DC005404002099A600085C04002030B597B068
:1041EC0002F0A2FE02F0C0FE09F08AF9554B002540
:1041FC004FF480301D7009F0A3F909F007FB01287A
:10420C00044627D1102009F02DFE022009F012FEE1
:10421C00284609F0E5F9284609F0F6F94FF48060D4
:10422C0009F0E8F94FF480304FF4E01109F0B4F9DB
:10423C00204609F0BDF9392009F0D2FA0028FAD04D
:10424C00022009F0BBF909F0C3F90828FBD13D4B5A
:10425C0001221A700120014609F078FA3A4C4FF409
:10426C0080414FF0006009F0D3FB4FF4407009F02F
:10427C0031FBFFF77DFF04F0E1FB04F019FC06F0C5
:10428C00CDFC03F069FA3149204604F0D1FD05F06C
:10429C00BDFA04F0E7FB207803F0A8FFE0782C4C83
:1042AC0003F010FF25460DF1100C0FCDACE80F00FC
:1042BC00AE46BEE80F00ACE80F009EE80F003034AD
:1042CC000DF1400E8CE80F000FCCAEE80F0094E817
:1042DC00030004248EE80300009404AC02221D4960
:1042EC0061230820019410AC029404F0D9FA00F078
:1042FC0039F800F031F800F0DDFC01F039FA02F089
:10430C00FFFD40F2127005F001FD40F2167005F051
:10431C009FFC02F025FF02F0A5FE00F033F820B957
:10432C0002F0A0FB00F036FC04E0012002F09AFB46
:10433C0000F046FD00F0C4FA02F0E4FD05F0BEFC0E
:10434C00E9E700BF6C0400208404002090030020E7
:10435C00A8F20008000C0140014B00221A707047B3
:10436C007C010020064B4FF448325A625A601A61A5
:10437C00DA619A605A611A62DA609A61704700BF1A
:10438C007C010020014B93F8280070477C01002031
:10439C00014B1868704700BFE4080020014BD86A35
:1043AC00704700BF7C01002008B5024B18680AF06A
:1043BC004FFF08BD1C090020014B186B704700BF54
:1043CC007C010020014B1868704700BF38090020A1
:1043DC00014B1868704700BFEC080020014B1868AF
:1043EC00704700BFF4080020034B93F8462022EAE4
:1043FC00000283F84620704790030020034B93F88B
:10440C00463018420CBF002001207047900300205A
:10441C00034B93F85D2040EA020283F85D2070475D
:10442C0090030020034B93F85D2022EA000283F8EE
:10443C005D20704790030020034B93F85D301842C9
:10444C000CBF00200120704790030020014B18681E
:10445C00704700BF08090020014B1868704700BF67
:10446C00D0080020014B5868704700BFD0080020CE
:10447C00014B1868704700BF20090020014B586899
:10448C00704700BF2009002008B50120FFF7D4FFBA
:10449C0048B1054B002204201A63FFF7CDFF10B181
:1044AC000120FFF7BFFF08BD7C01002008B505F017
:1044BC002DFE08BD08B505F095FC08BD08B54FF4F8
:1044CC00803004F08FFA08BD08B5044B93F86C30BB
:1044DC001BB94FF4003004F085FA08BD900300209E
:1044EC0008B5034B1B78012B01D103F023FE08BD4B
:1044FC004200002008B50220FFF780FF38B1044BC2
:10450C00B3F8440005F008FE0220FFF76DFF08BD6C
:10451C009003002008B50120FFF770FFC0B105F033
:10452C0005FE0C4991F825300A6C5B08B2FBF3F3DD
:10453C00B0FBF3F202FB1303074A21F8443F126865
:10454C0002F14400022204F0DFFA0120FFF74CFFD5
:10455C0008BD00BF900300200400002008B54FF4F4
:10456C00807009F0F1FC88B14FF4807009F0FAFC0E
:10457C00074B1B78012B03D0064B1B78012B05D165
:10458C00FFF7C8FFFFF7B6FFFFF77EFF08BD00BFC0
:10459C00400000201702002008B5044B19780129AF
:1045AC0003D1034B186808F04FFC08BD40000020F5
:1045BC003C00002038B5164C0221206808F03EFC67
:1045CC00012819D10221206808F03EFC002002F0DD
:1045DC00D5FD104C0546014694F8340005F0D2FB8D
:1045EC000D4B84F8345093F8213080B2062B03D154
:1045FC00226B03B29B182363054C0121206808F041
:10460C001DFC0128014602D1206808F01DFC38BDB4
:10461C00340000207C0100209003002008B5074BDB
:10462C001978012903D1064B186808F00DFC054BCD
:10463C001B78012B01D1FFF7BDFF08BD170200202D
:10464C003C0000201502002008B5074B1978012901
:10465C0003D1064B186808F0F7FB054B1B78012BB0
:10466C0001D1FFF7A7FF08BD160200203C00002077
:10467C003800002038B5204B93F82120062A02D0B0
:10468C00072A37D121E01D4A0128136B1B4D08BFA7
:10469C0093630128AA6B1A4CAB6302D1EB6B2360BA
:1046AC0028E09B1A144A206892F825104EF66022D6
:1046BC005343490806225143223293FBF1F106F091
:1046CC0003FC20602368EB6314E001280B4A0C4CBC
:1046DC0002D1136C23600AE00A490868196C4EF683
:1046EC006023434393FBF1F3236023681364054B6E
:1046FC0000221A6038BD00BF900300207C0100200E
:10470C00EC0800203409002010B504464FF480401A
:10471C0004F068F9034B01201C63DC62FFF7AAFF6D
:10472C0010BD00BF7C010020B0F5007F10B5044621
:10473C0010D003DCB0F5807F37D121E0B0F5806F6D
:10474C0003D0B0F5006F30D10DE004F043F94FF415
:10475C00807019E004F03EF94FF4807004F042F9D7
:10476C004FF4806014E004F035F94FF4807004F0DD
:10477C0039F94FF4806004F035F94FF400700BE018
:10478C0004F028F94FF4806004F02CF94FF4007019
:10479C0004F028F94FF4006004F024F94FF4804041
:1047AC0004F020F9024BA3F86E40024B1C6010BDC4
:1047BC0090030020F008002010B504464FF4803020
:1047CC0004F018F9012808D0044B4FF400601C6069
:1047DC00FFF7AAFF024B00221A6010BDF808002058
:1047EC001C09002038B505464FF4803004F002F95E
:1047FC0001281CD00E4B4FF480601C680D4BDD6201
:10480C00FFF792FF4FF4804004F0ECF8B4F5007F12
:10481C0004D1094B1A68094B1A6008E0B4F5006F13
:10482C0005D1074B18680AF0F9FA044B186038BD2B
:10483C00F00800207C0100201C090020B408002096
:10484C00EC08002008B5034B1B6BC018FFF7CAFF20
:10485C0008BD00BF7C01002038B505464FF4803000
:10486C0004F0C8F801281AD00D4B4FF400701C68E6
:10487C000C4B1D60FFF758FFB4F5006F05D10A4BC8
:10488C0018680AF0CBFA094B1860094B9B6813F4B3
:10489C00004F04D104F0C8F808B902F0F5FB38BD9C
:1048AC00F008002038090020EC0800201C0900202A
:1048BC000010014008B54FF48070FFF735FF08BDBC
:1048CC0010B504F09DFF1F4C636CC31A002BB8BFCE
:1048DC005B42B3F57A7F34DD1B4B9A6812F4006FA0
:1048EC0028D19B6813F4004F0CD0012004F072F80F
:1048FC00402004F06FF894F848300A2B02D80133AA
:10490C0084F848300020FFF7A7FF0F4B0F499A6837
:10491C00002012F4004F08600FD00A4A92F8482089
:10492C000A2A0AD84FF480621A6140205A6104F0B6
:10493C0059F802E0002384F8483004F061FF014B81
:10494C00586410BD7C010020001001401C0900209F
:10495C0038B5174B186808F069FA164B0422196C15
:10496C0091FBF2F290420ADA4FF0030C0CFB02FCC2
:10497C00114BDB6C634502DDCB1A1B180DE00323D6
:10498C005343984206DD0C4BDB6C934202DAC31A9C
:10499C005B1A02E0084BDB6CC31A074A0749146B1D
:1049AC000D68E41AEB1A0B60D064146338BD00BFB9
:1049BC003C000020900300207C01002034090020E2
:1049CC00214A10B51288214B12F0100F2CD11B78F4
:1049DC00012B03D11E4B4FF400521A611D491B4B86
:1049EC001D480C681A6D90F821000134013207281B
:1049FC000C601A6509D1132A04D9002210461A65D5
:104A0C00FFF738FE0120FFF7A3FF134B93F821307B
:104A1C00062B13D10D4B1A6D132A0FD900221046F9
:104A2C001A65FFF727FE09E01978012906D1084B12
:104A3C004FF4005209485A6109F004FF0248012161
:104A4C0008F002FA10BD00BF002C01407C010020D0
:104A5C0000100140CC0800209003002000240140ED
:104A6C0008B504F0CDFE194B5B6DC31A002BB8BF13
:104A7C005B42642B29DD164B93F82F30012B0CD1A4
:104A8C00144B186802F004FD40F6DD73984204D90B
:104A9C0002F002FB042003F09DFF0E4B186802F09D
:104AAC00F7FCB0F5FE6F02D2022003F093FF094B26
:104ABC00186802F0EDFCB0F5FE6F02D3022003F093
:104ACC0091FF04F09DFE014B586508BD7C01002050
:104ADC00900300202C00002010B504F091FE214B17
:104AEC009B6DC31A002BB8BF5B42FA2B39DD1E4BF2
:104AFC00186802F0CDFC0446082003F07BFFA0B937
:104B0C0040F6B3239C4207D9083003F063FF02F050
:104B1C00CBFA02F0C1FA20E0B4F5156F09D80820E1
:104B2C0003F060FF02F0C8FA08E040F60B239C4249
:104B3C0013D8082003F056FF02F0C6FA0B4B9B6803
:104B4C0013F4004F09D103F06FFF30B900F500509A
:104B5C0003F050FF08B902F097FA04F051FE014B34
:104B6C00986510BD7C010020300000200010014031
:104B7C0010B50224064A90FBF4F40346A4B2204676
:104B8C0082F8253005F0DAF8204605F081FA10BDE0
:104B9C0090030020F8B52E4B93F828201446002AD9
:104BAC0055D1DA6D25460132DA65012D03D0022D7F
:104BBC0003D0284B02E0284B00E0284B186802F089
:104BCC0067FC64274743264B1A59974201D9013297
:104BDC001A51244B1A59974201D2013A1A51214BBE
:104BEC0003F10C021E5912591833B6181B597608CA
:104BFC009E4201D95E1C01E038BF5E1E012D03D020
:104C0C00022D03D0134B02E0134B00E0134B642135
:104C1C001868B6FBF1F102F043FC124B12491A5919
:104C2C000E51BA4201D201321A510D4B1A59BA42E5
:104C3C0001D9013A1A5101350434032DB5D1044B75
:104C4C000A4AD96D914202DD012283F82820F8BD71
:104C5C007C010020100200202400002028000020ED
:104C6C008C01002080010020980100203F0D0300E2
:104C7C0010B50C4C23789BB90B4B4FF400611868A2
:104C8C0002F00EFC094B4FF40061186802F008FCAE
:104C9C00074B4FF40061186802F002FC01232370EB
:104CAC0010BD00BF7C010020100200202400002059
:104CBC002800002010B502F0B9F9012002F026FC02
:104CCC002F4C304803F0E2F92F4803F0DFF904F0E1
:104CDC004FFE94F82130062B0FD14FF4004003F017
:104CEC0079FE802003F07EFE012005F0EFF894F8A9
:104CFC002500400805F08EF801E005F0C7F8204CBF
:104D0C0094F82130072B21D14FF4004003F06AFEB8
:104D1C00802003F067FE94F82E30012B02D1002086
:104D2C0005F0D4F8164C206C94F8301005F054FAB9
:104D3C0094F82510206C490805F0B6F905F0C4F973
:104D4C0002F080FE012005F0C5F901E005F00EFA35
:104D5C00012002F0E1FB0D4B4FF480421A619B687D
:104D6C0013F4004F09D103F05FFE30B900F5005089
:104D7C0003F040FE08B902F087F9FFF779FF10BD88
:104D8C0090030020D00800202009002000100140D2
:104D9C0038B5094C094D94F8602095F821309A42A9
:104DAC0008D0FFF787FF0120FFF764FC95F821304E
:104DBC0084F8603038BD00BF7C01002090030020D7
:104DCC002DE9F0418EB004F01BFD4C4C0646636E91
:104DDC00C31A002BB8BF5B42B3F57A7F0DDB0025FD
:104DEC00A06E03F0C7FDE06EA56603F0C9FD206F51
:104DFC00E56603F0CBFD66662567414A3F4B1168BB
:104E0C00404A986E12690029B8BF49420130002A05
:104E1C00B8BF52429142986603DC102003F0DAFDD1
:104E2C0002E0102003F0DEFDFFF7B2FF354DFFF777
:104E3C0017FEFFF751FE344BAA6919689142C0F076
:104E4C0092802E4C0021226F4FF4004001321960E9
:104E5C00226703F0CFFD012822D14FF4806003F0CC
:104E6C00C9FD01281CD1E16A284B226B284603F0AE
:104E7C00EDF8E26A236B2649D21A002AEB68B8BF18
:104E8C0052429A4208600BDC1D4AAB681268002A39
:104E9C00B8BF52429A4203DC4FF4804003F09AFDB3
:104EAC00184C94F82030012B38D14FF4806003F06B
:104EBC00A1FD01280DD1114A1649136BD56A144A6C
:104ECC0020461268009502F023FD09F0A7FF124B53
:104EDC0018604FF4007003F08DFD012829D10E4CA1
:104EEC0020680AF0B5F90A4B01461A68054802F029
:104EFC00D9FC09F093FF20601BE000BF7C0100206F
:104F0C00EC080020900300203C0900200809002038
:104F1C0038090020B40800201C0900207F4B2168B0
:104F2C0018680A46494205F0AFFF09F077FF7C4B41
:104F3C0018604FF4007003F05DFD012805D04FF4AC
:104F4C00806003F057FD01280DD1764B1C68744B23
:104F5C0018680AF07DF9744B01462246734803F039
:104F6C0037F8734B1860734E704B3168DA699142A5
:104F7C00C0F04C81704F9A8DFB6E4FF0000EC6F84E
:104F8C0000E003F1010C1226C7F86CC00AAC0096C5
:104F9C006A4D06F5E876C8211423204601964FF495
:104FAC000266029602F024FB94E8070085E80700ED
:104FBC004FF4806003F01EFD01280BD04FF40070FD
:104FCC0003F018FD012805D04FF4006003F012FD2A
:104FDC00012830D1584C514B584A04F1740C6F468F
:104FEC0007CAD3F8008087E80700CDF814C0DFF8B3
:104FFC0068C14F4ECDF818C0DFF824C14FF0000E39
:10500C00494B4A484E494F4ACDF810E0CDF81CC0E8
:10501C00CDF82080039602F055FDB4F97430B4F944
:10502C007610494D3468C918484B286810221C600A
:10503C0005F04AFF2860444B3C4D1868294604F0A3
:10504C00A9FD04F0E1FD2B6E984225D904F0D8FBA4
:10505C00394CA36FC31A002BB8BF5B42B3F57A7FF0
:10506C001ADB04F08FFD4FF4003003F0B3FC95F81D
:10507C006C305BB9364B29461868012201F86C2F4D
:10508C006C3003F041FD04F0BBFBE06704F0CEFD97
:10509C0004F0B6FB284B986704F0B2FB264B23496F
:1050AC00DA6F4B6E821A002AB8BF52429A420BD367
:1050BC0091F86C20012A07D1254B1868002301F8C0
:1050CC006C3F6C3003F020FD184B93F86C30012BC7
:1050DC0003D14FF4003003F07DFC4FF4003003F0AB
:1050EC0089FC012808D1104802F0D0FF194802F0C1
:1050FC00CDFF0020FFF760FB02F052FA124B1A684A
:10510C000A4B002A5B68B8BF52429A4226DD012046
:10511C0003F060FC01F0E6FF25E000BF3809002039
:10512C001C090020EC080020D0080020900300206F
:10513C00F8080020CC0800207C010020FC0800208E
:10514C0020090020B8080020F4080020E408002002
:10515C000400002008090020B4080020012003F0FE
:10516C0041FC01F0C7FF2B4B93F8222012F0010FEA
:10517C0022D0294A1268002A1EDD93F8233013F03E
:10518C00010F03D0002001F0BDFF40B9214B93F873
:10519C00230010F001000FD101F0B4FF60B9022020
:1051AC00FFF74AF910B11D4B00221A630020FFF7DC
:1051BC0053FB1B4B00221A60164B93F8222012F063
:1051CC00020F23D0144A1268002A1FDA93F82330F6
:1051DC0013F0020F03D0012001F094FF48B90D4BDE
:1051EC0093F8233013F0020F10D1012001F08AFF45
:1051FC0060B90220FFF720F910B1084B00221A63A6
:10520C000020FFF729FB064B00221A600EB0BDE808
:10521C00F08100BF90030020EC0800207C010020EE
:10522C001C0900200A4938B50C6B0023CC620949D3
:10523C00094D0B60094900220A602A60084A094D91
:10524C0001202B601360FFF715FAFFF733FD38BD13
:10525C007C010020380900201C090020B408002023
:10526C00E4080020F808002010B5104B5B788BB9CF
:10527C000F4A012091780F4A14680F4A10700F4A98
:10528C0011700133E21812F8011C0C4A082B9954C6
:10529C00F7D109E0012B07D1094B06210222D97164
:1052AC0062311A7199715A7110BD00BF1803002038
:1052BC0084040020180000208003002084030020B8
:1052CC0074040020044B5A6840F2D2439A4202D133
:1052DC00024B01221A70704718030020400900206D
:1052EC0010B51A4A1A4B116801EA030319498B428B
:1052FC002AD15268184B9A4226D101F0CDFE03F008
:10530C007FFA04F07DFA044601E001F0ABFE04F0F4
:10531C0077FA001B0028B8BF4042B0F57A7FF4DB67
:10532C0003F08EFB08F0A4FA002007F029FF0021FF
:10533C000A4808F0BDFE094808F01AFE084809F0B2
:10534C00C1FB002003F086FB10BD00BF180300203A
:10535C0000FFFF0000819200D6C5B4A308000240F4
:10536C000024014010B5164B9A78012A08D003D3BB
:10537C00022A144C0FD109E0587801F0C3FE02E068
:10538C00587801F0EFFE0F4B586006E0587801F0AA
:10539C00C9FE606001E0042323700B4B1B786BB1DA
:1053AC00084B0A495A680A4B0A601AB91A6842F043
:1053BC00080202E01A6822F008021A6010BD00BF51
:1053CC001803002074040020580400207C030020E3
:1053DC002003002008B5104B9A78012A02D0022A2B
:1053EC0016D10CE05A7842B9586810B903F02AFB70
:1053FC0011E0104603F02AFB0DE0032209E05A6885
:10540C00587812B901F030FE05E001F035FE02E0EB
:10541C000422024B1A7008BD1803002074040020EB
:10542C0008B50B4B9A78022A0ED15B78372B09D82A
:10543C009B00084903F5E260C9180A30023203F0F8
:10544C003FFB04E0032200E00422034B1A7008BD6A
:10545C0018030020B00400207404002008B58F4B02
:10546C009A78002A40F074815B78A62B00F0C180FA
:10547C002BD81A2B00F08D8011D8092B71D007D89E
:10548C00062B62D0072B66D0042B40F05F8157E0CF
:10549C000B2B72D06BD3192B40F0588173E09F2BE0
:1054AC0000F08F8008D8862B7FD0922B00F0838061
:1054BC00852B40F04B8172E0A42B00F08E8000F223
:1054CC009280A12BC0F0428181E0F02B00F0C780CC
:1054DC001CD8E62B00F0A58009D8AD2B00F09580E8
:1054EC00B12B00F09880AC2B40F0308187E0EB2B97
:1054FC0000F0A38003D8EA2B40F0288197E0EE2B34
:10550C0000F0A180EF2B40F02181A2E0F92B00F0FC
:10551C00BE8009D8F42B00F0AE80F52B00F0B180E2
:10552C00F12B40F01381A0E0FB2B00F0FB80C0F0CE
:10553C00F380FD2B00F0FC80FE2B40F00781FDE09A
:10554C00574B584918680422FDE0554B0422186843
:10555C0055498018F7E0524B54491868042208301A
:10556C00F1E04F4B5249186804221030EBE04C4BE1
:10557C005049186804220C30E5E0494B4E49186834
:10558C0004221430DFE0464B4C4918680422643086
:10559C00D9E0434B4A49186804226030D3E0404BB1
:1055AC004849186804221830CDE03D4B464918682C
:1055BC0004221C30C7E03A4B4449186801222030C1
:1055CC00C1E0374B4249186801222130BBE0344B13
:1055DC004049186801225D30B5E0314B3E491868EE
:1055EC0001222230AFE02E4B3C4918680222443095
:1055FC00A9E02B4B3A49186801222330A3E0284B31
:10560C0038491868042234309DE0254B3649186817
:10561C000422383097E0224B3449186804223C307D
:10562C0091E01F4B32491868042250308BE01C4B20
:10563C00304918680422543085E0194B2E491868FB
:10564C00042258307FE0164B2C491868042228306D
:10565C0079E0134B2A4918680422483073E0104B48
:10566C002849186804224C306DE00D4B2649186807
:10567C000422683067E00A4B24491868022226305D
:10568C0061E0074B2249186801222F305BE0044B84
:10569C002049186801222E3055E000BF1803002065
:1056AC0004000020900300209403002098030020A5
:1056BC00A00300209C030020A4030020F40300207E
:1056CC00F0030020A8030020AC030020B00300204E
:1056DC00B1030020ED030020B2030020D40300200E
:1056EC00B3030020C4030020C8030020CC03002017
:1056FC00E0030020E4030020E8030020B8030020AE
:10570C00D8030020DC030020F8030020B60300209F
:10571C00BF030020BE0300200F4B10491868042261
:10572C00403010E00C4B0E491868012230300AE072
:10573C00094B0C4918680122253004E0064B0A4934
:10574C0018680122243003F0BBF904E0032200E0C6
:10575C000422064B1A7008BD04000020D003002060
:10576C00C0030020B5030020B40300207404002003
:10577C00144A00231360144A10B51360134A1360C3
:10578C00134A1360134A1370134A002199500433BF
:10579C00B3F5806FF8D1114B1B7E63B940F21A74CC
:1057AC000F4920460919042203F08AF9043440F207
:1057BC00FA739C42F4D1094A0A4B527D02B1012280
:1057CC001A7010BD200400207C030020AC040020C3
:1057DC002003002014030020B004002084040020C7
:1057EC0096FDFF1F6004002008B50B4B9A78022A27
:1057FC000ED15B78372B09D89B00084903F5E26082
:10580C00C9180A30023203F07FF904E0032200E0E9
:10581C000422034B1A7008BD18030020B0040020AA
:10582C007404002008B5604B9A781AB1022A40F033
:10583C00A68099E05B78502B69D020D8452B51D0AD
:10584C000ED8422B44D005D8402B38D0412B40F0F9
:10585C0089803BE0432B3FD0442B40F083803EE0DB
:10586C00492B48D004D8462B3FD0472B7AD13FE068
:10587C004C2B46D04D2B47D04B2B73D13EE0812B7C
:10588C0059D00ED8532B4BD004D8512B42D0522B7D
:10589C0068D142E05A2B49D0802B4AD0552B61D18C
:1058AC0041E0842B52D004D8822B4BD0832B59D17E
:1058BC004AE0FE2B4DD04FD8F02B53D149E03B4B57
:1058CC00186803F09FF93A4B58605BE0394B41E0A4
:1058DC00384B5A78364B4EE0364B1A79FAE7354B43
:1058EC00DA69F7E7334B5A79F4E7324BDA68F1E7C8
:1058FC00304B9A68EEE72F4BDA7D2FE02D4BDA78A0
:10590C00E8E72C4B9A78E5E72A4B5A7DE2E7294BDE
:10591C009A7DDFE7274B1A7DDCE7264B1A6AD9E71D
:10592C00244B1A69D6E7234B1A7ED3E7214B5A6ACC
:10593C00D0E7214B0EE0204B1A78042A14BF00222A
:10594C000122C7E71D4B02E01D4B00E01D4B1A68FE
:10595C00C0E71D4B1A78BDE71C4B1A78003A18BFEC
:10596C000122B7E703220BE05A78114B372A04D8EF
:10597C00174951F822205A6004E0032201E0042266
:10598C000B4B1A70134B1B786BB1094B12495A68AD
:10599C00124B0A601AB91A6842F0080202E01A683F
:1059AC0022F008021A6008BD180300200C00002029
:1059BC0074040020840400206004002020040020D3
:1059CC0048090020440900206C04002050040020E9
:1059DC00B0040020580400207C0300202003002089
:1059EC0010B5884B9A781AB1022A40F01D81FEE05E
:1059FC005A784C2A00F09C801ED8442A5ED00CD8D1
:105A0C00412A42D003D8402A40F0F98039E0422A9A
:105A1C0044D0432A40F0F38048E0472A66D005D8AA
:105A2C00452A53D0462A40F0EA8057E0492A65D0EF
:105A3C004B2A40F0E4806EE0532A00F0AD800ED883
:105A4C00502A00F0858003D84D2A40F0D88077E0AA
:105A5C00512A00F08580522A40F0D18094E0832AAC
:105A6C0000F0B98006D8552A00F09E805A2A40F0E2
:105A7C00C680A5E0842A00F0B280FF2A40F0BF80E7
:105A8C00B2E01979604B186805E0604A1B79106820
:105A9C005F4A1946137003F0CDF8C8E05B4A1B79D6
:105AAC0010685B4A013019465370F4E7574A1B796A
:105ABC001068574A043019461371ECE7534A5B6877
:105ACC00106853491C3041F81C3F80E04F4A1B7949
:105ADC0010684F4A053019465371DCE74B4A5B6836
:105AEC0010684B490C3041F80C3F70E0474A5B683A
:105AFC0010684749083041F8083F68E01A79444B70
:105B0C0012B1444901224A60DA75404B1868404B87
:105B1C001730D97DBFE73D4A1B7910683C4C0330E8
:105B2C001946E37003F086F8E07802F0CBFA7EE0D9
:105B3C00364A1B791068364A023019469370AAE728
:105B4C00324A1B791068324A153019465375A2E750
:105B5C002E4A1B7910682E4A1630194693759AE70F
:105B6C002B4A127D12F0010F05D01B7913F0010F97
:105B7C0001D103F017F9254A224B10681B79244AEE
:105B8C0014301946137586E7204A5B681068204963
:105B9C00203041F8203F1AE01C4A5B6810681C4911
:105BAC00103041F8103F12E05A68012A3CD8174ACD
:105BBC001B7910681649183001F8183F012207E0CC
:105BCC00124A5B6810681249243041F8243F0422C1
:105BDC0002F09AFF2BE00F4B5A680F4B02E00D4B73
:105BEC005A680E4B1A6022E01A790D4B1EE05A7857
:105BFC00372A04D859680B4B43F8221017E00322BC
:105C0C0013E000BF180300200C00002078010020D6
:105C1C00840400207404002048090020440900205A
:105C2C0050040020B00400200422014B1A7010BD57
:105C3C007404002008B58F4B9A78002A40F07C81C0
:105C4C005B78A52B00F0C7802FD81C2B00F0998017
:105C5C0013D8092B77D007D8062B68D0072B6CD01C
:105C6C00042B40F067815DE00B2B78D071D3192B9E
:105C7C007BD01A2B40F05E817DE0922B00F093805C
:105C8C0009D8852B00F08380862B00F086801E2B94
:105C9C0040F0508178E0A32B00F29780A12B80F08C
:105CAC008E809F2B40F0468183E0EF2B00F0C98063
:105CBC001CD8B12B00F0A78009D8AC2B00F0978032
:105CCC00AD2B00F09A80A62B40F0348189E0EA2BB2
:105CDC0000F0A58003D8E62B40F02C8199E0EB2B4B
:105CEC0000F0A380EE2B40F02581A4E0F92B00F00E
:105CFC0001810BD8F12B00F0B080C0F0A880F42B00
:105D0C0000F0B180F52B40F01581EDE0FB2B00F09D
:105D1C00FD80C0F0F580FD2B00F0FE80FE2B40F0E6
:105D2C000981FFE0544B554918680422FFE0524B9F
:105D3C000422186852498018F9E04F4B51491868F1
:105D4C0004220830F3E04C4B4F4918680422103001
:105D5C00EDE0494B4D49186804220C30E7E0464B06
:105D6C004B49186804221430E1E0434B4949186848
:105D7C0004226430DBE0404B474918680422603051
:105D8C00D5E003F053FFDAE003F080FFD7E03A4BA5
:105D9C004249186804221830C9E0374B404918684A
:105DAC0004221C30C3E0344B3E49186801222030D9
:105DBC00BDE0314B3C49186801222130B7E02E4B35
:105DCC003A49186801225D30B1E02B4B384918680C
:105DDC0001222230ABE0284B3649186802224430AD
:105DEC00A5E0254B34491868012223309FE0224B53
:105DFC00324918680422343099E01F4B3049186836
:105E0C000422383093E01C4B2E49186804223C3095
:105E1C008DE0194B2C4918680422503087E0164B42
:105E2C002A4918680422543081E0134B2849186819
:105E3C00042258307BE0104B264918680422283085
:105E4C0075E00D4B24491868042248306FE00A4B6A
:105E5C002249186804224C3069E0074B2049186825
:105E6C000422683063E0044B1E4918680222263075
:105E7C005DE000BF18030020040000209003002008
:105E8C009403002098030020A00300209C03002012
:105E9C00A4030020F4030020F0030020A80300203A
:105EAC00AC030020B0030020B1030020ED03002060
:105EBC00B2030020D4030020B3030020C40300204D
:105ECC00C8030020CC030020E0030020E4030020E2
:105EDC00E8030020B8030020D8030020DC030020D6
:105EEC00F8030020B6030020154B16491868012250
:105EFC002F301CE0124B1449186801222E3016E08A
:105F0C000F4B124918680422403010E00C4B10491A
:105F1C001868012230300AE0094B0E49186801223A
:105F2C00253004E0064B0C4918680122243002F09D
:105F3C00EBFD04E0032200E00422084B1A7008BDBC
:105F4C0004000020BF030020BE030020D00300206B
:105F5C00C0030020B5030020B4030020740400200B
:105F6C0010B5A34B9A78002A40F0B6815B78AC2B25
:105F7C0000F0378163D81E2B00F0F4802ED8092B4B
:105F8C0000F0D88014D8032B00F0C88006D8012B61
:105F9C0000F0BE80974C00F2BE80B6E0062B00F0FD
:105FAC00C380072B00F0C380042B40F09381B8E032
:105FBC00192B00F0CB8008D80B2B00F0C180C0F05F
:105FCC00BC800D2B40F08681BDE01B2B00F0C48003
:105FDC00C0F0BF801C2B40F07D81C0E09C2B00F0FA
:105FEC00DB8016D8962B00F0CA8009D8862B00F0DF
:105FFC00BF80922B00F0BF80852B40F06B81B4E00A
:10600C00982B00F0C180C0F0BD809B2B40F06281CA
:10601C00BFE0A32B00F0D38008D8A12B00F0C380E5
:10602C0000F2C7809F2B40F05581B8E0A52B00F003
:10603C00D080C0F0CA80A62B40F04C81CDE0E42B80
:10604C0000F00B812FD8C32B00F0EF8014D8BF2B9E
:10605C0000F0DE8009D8B12B00F0D480BE2B00F00C
:10606C00D480AD2B40F03681BEE0C12B00F0D68041
:10607C00604C00F2D680CEE0C92B00F0E28008D84C
:10608C00C52B00F0D880C0F0D380C82B40F0228103
:10609C00D4E0D32B00F0DB80E22B00F0DB80D22BA2
:1060AC0040F01881D0E0F12B00F0F18015D8EB2BEB
:1060BC0000F0E18008D8E62B00F0D780C0F0D0804B
:1060CC00EA2B40F00781D3E0EF2B00F0DA8000F2EE
:1060DC00DB80EE2B40F0FE80D0E0FA2B00F0E68067
:1060EC0009D8F52B00F0DA80F92B00F0DB80F42BCB
:1060FC0040F0F080CEE0FD2B00F0DF80FE2B00F0B6
:10610C00E080FB2B40F0E680D3E0FEF747F98AE015
:10611C00FEF752F9A6E0FEF755F984E0FEF758F9C0
:10612C00A0E0354B1A68D2E0334B5A68CFE0324BC3
:10613C009A68CCE0304B1A69C9E02F4BDA68C6E09C
:10614C002D4B5A69C3E0FEF72FF98BE02A4B5A6EA0
:10615C00BDE0294B1A6EBAE003F056FD82E003F065
:10616C0059FD7FE003F086FD7CE0234B9A69AEE09D
:10617C00214BDA69ABE0204B93F82020A4E0FEF72A
:10618C002DF96FE01D4B00E01D4B186801F080F9F4
:10619C0068E0FEF7FDF865E002F03CFC62E0164BAF
:1061AC0093F8212093E0144B93F85D2002F0010248
:1061BC008DE0114B93F85D20C2F3400287E00E4B4B
:1061CC0093F85D20C2F3800281E00B4B93F8222000
:1061DC007DE0094BB3F8442079E0074B93F823207A
:1061EC0075E0054B5A6B72E0034B9A6B6FE000BF86
:1061FC001803002074040020900300202C000020C1
:10620C00300000203F4BDA6B61E002F083FB29E0A9
:10621C0002F086FB26E002F089FB04E002F08CFB26
:10622C0020E002F08FFB606059E002F091FB19E076
:10623C0002F094FB16E002F097FB13E0FEF718F95E
:10624C0010E0FEF71BF90DE0FEF734F90AE0FEF75B
:10625C002DF907E0FEF7FAF804E0FEF7FDF801E08F
:10626C00FEF700F9284B586039E0264B1A6D2EE0EA
:10627C00244B5A6D2BE0234B9A6D28E0214B9A6AE4
:10628C0025E0204B9A6C22E01E4BDA6C1FE01D4B74
:10629C009A6E1CE01B4BB3F9262018E0194B93F8AF
:1062AC002F2011E0174B93F82E2010E0154B1A6C91
:1062BC000DE0144B93F8302006E0124B93F8252098
:1062CC0005E0104B93F82420003A18BF01220E4B26
:1062DC005A6004E0032200E004220B4B1A700B4BB3
:1062EC001B786BB1084B0A495A680A4B0A601AB9F9
:1062FC001A6842F0080202E01A6822F008021A60DA
:10630C0010BD00BF9003002074040020580400202E
:10631C007C0300202003002008B50020FEF79CFA27
:10632C0008BD00BF08B5024B5868FEF795FA08BDCA
:10633C001803002008B5034B58684042FEF78CFA4E
:10634C0008BD00BF1803002008B59A4A9378002BAB
:10635C0040F0EE815378A52B00F0548156D81D2BBC
:10636C0000F0E8802AD8072B00F0C38011D8022B4C
:10637C0000F0B18006D8002B00F0A380012B40F078
:10638C00D581A3E0042B00F0AA80062B40F0CE812F
:10639C00AAE00B2B00F0BB8006D8092B00F0AD80D7
:1063AC000A2B40F0C381ADE01A2B00F0B9801C2BF6
:1063BC0000F0BB80192B40F0B981ACE09B2B00F0B6
:1063CC00D78011D8852B00F0C08006D81E2B00F08A
:1063DC00B4801F2B40F0AA81B4E0862B00F0B9806A
:1063EC00922B40F0A381B9E0A12B00F0D38006D80A
:1063FC009E2B00F0C1809F2B40F09881BFE0A32B17
:10640C0000F0E9806B4B00F2F480D7E0E62B00F053
:10641C003E8129D8BF2B00F0178111D8AD2B00F08D
:10642C00058106D8A62B00F0F280AC2B40F07E81C3
:10643C00F7E0B12B00F0FE80BE2B40F07781FEE040
:10644C00C22B00F0108106D8C02B00F00281C12BAA
:10645C0040F06C8102E1C42B00F00F81C0F0088188
:10646C00C52B40F063810DE1F42B00F0318113D882
:10647C00EE2B00F01A8106D8EA2B00F00C81EB2BE6
:10648C0040F054810CE1F02B00F01881C0F0118128
:10649C00F12B40F04B8116E1FA2B00F02C8106D841
:1064AC00F52B00F01981F92B40F040811DE1FD2BFB
:1064BC0000F02E81FE2B00F03081FB2B40F036815A
:1064CC001DE13C4B5868FEF78DF934E1394B5868A7
:1064DC00FEF71AF92FE15068FEF7BEF92BE1354BA8
:1064EC005A68354B1A6026E1324B5A68324B5A6067
:1064FC0021E15268304B9A601DE12E4B5A682E4BAD
:10650C001A6118E12B4B5A682B4BDA6013E1526875
:10651C00294B5A610FE1274B5A68274B5A660AE1FF
:10652C00244B5A68244B1A6605E1224B586803F039
:10653C0077FB00E1FDF7C8FFFDE01E4B586803F048
:10654C009FFBF8E0FEF76EFEF5E052681A4B9A617D
:10655C00F1E0184B5A68184BDA61ECE0154B5A68AD
:10656C00012A00F2E5801A79134B83F82020E2E02F
:10657C005068FEF721F9DEE0FDF7A0FFDBE00D4BE4
:10658C005A68063A012A00F2D3801A790A4B83F82A
:10659C002120D0E05268084B22B193F85D2042F0E4
:1065AC00010203E093F85D2022F0010283F85D20E4
:1065BC00C1E000BF18030020900300205A685E4B16
:1065CC0022B193F85D2042F00202EFE793F85D20D0
:1065DC0022F00202EAE7594A574B526822B193F86B
:1065EC005D2042F00402E1E793F85D2022F0040202
:1065FC00DCE75A68032A00F29B801A794E4B83F829
:10660C00222098E04C4B9288A3F8442093E04B4B0B
:10661C005A68032A00F28C801A79474B83F823209E
:10662C0089E0464B5A68444B5A6384E05268424BAB
:10663C009A6380E0414B5A683F4BDA637BE0404BF6
:10664C00586802F097F976E03D4B586802F098F9DB
:10665C0071E03B4B586802F099F96CE0384B586884
:10666C0002F09AF967E0364B586802F09BF962E049
:10667C00334B586802F09CF95DE0314B586802F0DE
:10668C009DF958E02E4B586802F09EF953E0526881
:10669C00294B1A654FE0294B5A68274B5A654AE03B
:1066AC00264B5A68244B9A6545E05268224B9A62F5
:1066BC0041E0224B5A68204B9A643CE01F4B5A68CD
:1066CC001D4BDA6437E01D4B5A681B4B9A6632E05F
:1066DC00194B9288DA842EE0184B5A68164B003A04
:1066EC0018BF012283F82F2025E0144B5A68124B57
:1066FC0083F82E201FE052680F4B1A641BE00F4BDF
:10670C005A680D4B003A18BF012283F8302012E072
:10671C000A4B5868FEF72CFA0DE0084B5A68064BEA
:10672C00003A18BF012283F8242004E0032200E081
:10673C000422034B1A7008BD90030020180300209C
:10674C007404002008B50B4B9A7872B95A7812B1C0
:10675C00012A08D103E05868FEF744F808E05868AD
:10676C00FEF770F804E0032200E00422024B1A70DA
:10677C0008BD00BF180300207404002010B5AA4BFC
:10678C00AA4A59681B7851606421212B11705370EF
:10679C0000F0FD8057D80E2B00F0D28029D8062BA4
:1067AC0000F0B98011D8032B00F0AC8006D8012B77
:1067BC0000F0A280022B40F04F81A0E0042B00F0EF
:1067CC00A480052B40F04881A2E0092B00F0AC809E
:1067DC0006D8072B00F0A280082B40F03D81A0E0EA
:1067EC000B2B00F0A780C0F0A2800C2B40F0348162
:1067FC00A3E0172B00F0B68011D8142B00F0A98061
:10680C0006D80F2B00F09F80132B40F025819DE0C4
:10681C00152B00F0A180162B40F01E819FE01C2B45
:10682C0000F0A98006D8182B00F09F801B2B40F09D
:10683C0013819DE01F2B00F0A48000F2A5801E2B7D
:10684C0040F00A819AE0802B00F0C88029D8412BB7
:10685C0000F0AF8011D8242B00F0A28006D8222B98
:10686C0000F09880232B40F0F78096E0272B00F067
:10687C009A80402B40F0F08098E0442B00F0A280EE
:10688C0006D8422B00F09880432B40F0E58096E030
:10689C00462B00F09D80C0F09880472B40F0DC80A8
:1068AC0099E0872B00F0C68011D8832B00F09F80D5
:1068BC0006D8812B00F09580822B40F0CD8093E0A0
:1068CC00852B00F0A1805A4C00F2A68092E08C2B14
:1068DC0000F0B68006D8882B00F0A380892B40F0FE
:1068EC00BB80AAE0F22B00F0B180FF2B00F0B1804E
:1068FC008D2B40F0B180A6E0FFF714FDAFE0FFF761
:10690C0019FDACE0FFF708FDA9E0FFF71BFFA6E0BF
:10691C00FFF71AFDA3E0FFF723FBA0E0FFF78AF9CE
:10692C009DE0FEF79BFD9AE0FFF75AF897E0FEF723
:10693C0079FF94E0FEF758FF91E0FEF771FD8EE0D1
:10694C00FEF748FD8BE0FEF70DFD88E002F096FBAC
:10695C0085E002F071FC82E002F0FCFC7FE002F0CA
:10696C00EFFC7CE002F050FD79E002F065FD76E092
:10697C0002F0DCFD73E002F071FD70E002F074FDDA
:10698C006DE002F089FD6AE002F0B6FD67E002F00E
:10699C00C9FB64E002F0EEFE61E002F0DFFE5EE0B7
:1069AC0002F01EFC5BE002F0C3FA58E000F0ACFA17
:1069BC0055E000F0ABFA52E000F0AAFA4FE000F01C
:1069CC00A9FA4CE000F0A8FA49E000F0A7FA46E07A
:1069DC0000F0A6FA43E000F0A5FA40E002F0F8FA65
:1069EC003DE002F0BFFA3AE002F0CEFA37E002F0F6
:1069FC00D1FA34E000F050FB247D02F00BF8014694
:106A0C00204602F045FC2AE002F05EFC00F03CFB64
:106A1C000020FDF7D1FE22E0217DA07802F03CFEA3
:106A2C001DE0FEF721FC1AE018030020740400207E
:106A3C008404002002F04EFC11E002F073FE0EE024
:106A4C0002F0FEFD0BE002F0C9FA08E0FEF748FC8C
:106A5C0005E0FEF737FC02E0014B02221A7010BD74
:106A6C0074040020F0B5924B87B01B78044663B1D8
:106A7C00904B1B78062B08D00A2B06D00F2B04D07A
:106A8C001F2B02D08C4B00221A708B4B1B78032BC4
:106A9C0020D18A4B1B7893B9894E8A4DB078777880
:106AAC002A786B78C719BF18EA79FF18AB79BF1829
:106ABC006A79FF182B79BF18FF18FFB219E0012B68
:106ACC0031D10025804BE85C013501F00BFB092D21
:106ADC00F8D128E0042B26D1794E7A4DB37877780B
:106AEC001846DF190137002301222A706B60FFB2B0
:106AFC006B7001F0F7FA707801F0F4FA287801F075
:106B0C00F1FA687801F0EEFAE87901F0EBFAA8797D
:106B1C0001F0E8FA687901F0E5FA287901F0E2FA77
:106B2C00384601F0DFFA644B1B78072B35D1634BE9
:106B3C001B782BBB624A634B5578967893F800E030
:106B4C0093F801C0AF19D8797744997967445A7989
:106B5C00C7191B79CF19D719DF198DF808708DF863
:106B6C0000608DF801508DF802E08DF803C08DF8AF
:106B7C0004008DF805108DF806208DF8073009E01B
:106B8C00012B07D1013B504A995C0DF803100133DE
:106B9C00092BF8D16846092124E0082B24D1484A56
:106BAC00484B92F801C092F802E001250EEB0C065E
:106BBC0000220136684609215A608DF802508DF882
:106BCC00032017468DF804208DF805208DF806203B
:106BDC008DF807208DF808605A701D708DF800E054
:106BEC008DF801C001F0F6FC384B34491A780023BB
:106BFC000B7031490B7012B1012001F02BFF0DF11C
:106C0C00170001F049FA054600286CD001F060FA33
:106C1C0010B1294B00225A70274B9DF81700597858
:106C2C004A1CD2B2C918092A08715A705AD1244A7E
:106C3C0018795178002288425A7053D113461E4D50
:106C4C00291D895C01325B18082ADBB2F7D12A7B3B
:106C5C009A4245D1174B697AAA7AEE7A6F7995F8F0
:106C6C0006E095F807C0287A1E7199715A711F7049
:106C7C0083F801E083F802C0D87102F0C1FD144B17
:106C8C00144E1B783060591E13480022C9B26A702A
:106C9C000270033201292A7005D9052B03D00F4B42
:106CAC0001251D701FE00D4B00221A701AE000BF69
:106CBC005004002018030020000200208003002054
:106CCC008404002074040020840300204009002068
:106CDC0060040020700400207C0400205804002074
:106CEC0004232B70012503A801F05CFC002844D080
:106CFC00534B9DF80C205B789A4259D100221346D5
:106D0C0003A9C95C01335218082BD2B2F8D19DF8F3
:106D1C0014104C4C91422ED14B4B9DF811109DF8F8
:106D2C0012209DF80D609DF80EE09DF80FC09DF8A7
:106D3C0010009DF8135099715A711E701D7183F8D3
:106D4C0001E083F802C0D87102F05AFD3F4B404974
:106D5C001B7808605A1E3F490020D2B208700721E8
:106D6C00012A217003D9052B01D0012200E0002259
:106D7C00394B1A701CE023701AE0CDB933490B78EB
:106D8C00013BDBB2012B13D8012C11D1334B1A6808
:106D9C00B2F5006F0BD8104601321A602A4902F086
:106DAC0085F8284B09221A702B4B1C7000E00D70D3
:106DBC00264B1B78042B04D1234B93F90030002B6A
:106DCC002EDA204B1B783BB1042B05D0082B03D0BB
:106DDC00062B01D0FFF7D2FC1A4B1B78092B05D1DF
:106DEC001A4A1178022901D1033111701C4A126818
:106DFC001AB3092B21D1154B1B78012B1DD1174927
:106E0C00013B096809E0174850F82300013381421F
:106E1C0003D10E4B05221A700FE09342F3D30CE012
:106E2C00FDF748FD074B1B783BB1042B05D0082B15
:106E3C0003D0062B01D002F0D9FB07B0F0BD00BF88
:106E4C0084040020000200201803002060040020AD
:106E5C00700400207C040020580400202004002032
:106E6C00640400202404002073B5204B02464078B3
:106E7C001F4D1870907800265870D078EC4698709A
:106E8C0010790C46D8715079987192F806E095E813
:106E9C00030083F805E0D2798CE803001A71154BD6
:106EAC001E70FFF76BFC144B1B7873B96370237067
:106EBC002B78A3706B78E370EB792371AB796371EA
:106ECC006B79A3712B79E37108E0012B06D10B4B85
:106EDC009B195B78A3550136082EF8D1044B6A46F2
:106EEC0092E8030083E803007CBD00BF1803002078
:106EFC007404002058040020800300208403002028
:106F0C00704700BF704700BF704700BF704700BF9D
:106F1C00704700BF704700BF704700BF704700BF8D
:106F2C00704700BF704700BF0E4B10B50022012008
:106F3C0002214FF4FA744FF0080C5C6283F805C020
:106F4C009860D9601A621A7058709970DA701A7158
:106F5C009A711A611A755A759A75DA751A76DA6118
:106F6C0010BD00BF84040020284BF0B54FF4FA7715
:106F7C009F604FF4FA675F614FF0060C0227DF61E8
:106F8C0083F821C0BC44C6379F6640F2DC574FF4EF
:106F9C007A65DF63A7F59667002201204FF416741B
:106FAC0005261D641F651D605D6007F5FA774FF4BB
:106FBC007A75DA6483F8222083F8232083F824205E
:106FCC009A629A8583F82F2083F83020A3F8442006
:106FDC0083F846201E6183F825C05F659C6583F8A5
:106FEC005C00DE60986183F82000DD8483F82E005D
:106FFC005C639C639A6483F85D2083F86C20044A7C
:10700C001A6643F290325A66F0BD00BF900300201E
:10701C0000390300014B10225A61704700080140EF
:10702C00014B10221A61704700080140024B4FF4CB
:10703C0080521A61704700BF00100140024B4FF4A0
:10704C0080525A61704700BF00100140704700BF6A
:10705C00704700BF704700BF704700BF704700BF4C
:10706C00704700BF704700BF18B9024B4FF4007255
:10707C005A6170470010014018B9024B4FF400726E
:10708C001A61704700100140024B4FF400421A6124
:10709C00704700BF00100140024B4FF400425A6190
:1070AC00704700BF00100140024B4FF480521A6130
:1070BC00704700BF000C0140024B4FF480525A61E4
:1070CC00704700BF000C0140054B9A6812F4805FBA
:1070DC0015BF4FF480524FF480525A611A617047B9
:1070EC00000C0140024B4FF400721A61704700BF54
:1070FC00000C0140024B4FF400725A61704700BF04
:10710C00000C014018B1012803D0002005E0034B0E
:10711C0000E0034B9868C0F38000704700140140F6
:10712C00000C014008B1002003E0024BD868C0F30A
:10713C004020704700100140014B20221A6170471B
:10714C00000C0140014B20225A617047000C014099
:10715C00024BD86800F02000704700BF000C0140C3
:10716C00704700BF08B508B1002003E0024B186857
:10717C0000F08EF908BD00BF14000020094B10B5BB
:10718C009C6814F0070401D0072C05D1012803D109
:10719C001F3001F01FFC02E0202001F023FC2046F0
:1071AC0010BD00BF0008014037B501AD00242946D1
:1071BC004FF01F030848ADF804308DF8074006F077
:1071CC0005FD4FF00103294604488DF80740ADF842
:1071DC00043006F0FBFC3EBD00100140000C0140E9
:1071EC002DE9F745484F01AD04200121032406F099
:1071FC00ADFA4FF01008384629464FF0B803ADF8F9
:10720C0004308DF806408DF8078006F0DFFCA823CB
:10721C000426DFF8FCA0C7F81080384629467B61AD
:10722C004FF04703ADF804308DF806408DF8076039
:10723C0006F0CCFC0820012106F088FA50462946BD
:10724C0041F23A23ADF804308DF806408DF80780F2
:10725C0006F0BCFC4FF40E73CAF8143002235046EF
:10726C002946CAF8103040F6C55307F50067ADF84B
:10727C0004308DF806408DF8076006F0A7FC4046F8
:10728C00012106F063FA384629464FF20063ADF847
:10729C0004308DF807808DF8064006F097FC4FF40B
:1072AC00E4433B6103F59153384629467B614FF427
:1072BC001E63ADF804308DF806408DF8076006F0BB
:1072CC0085FC4FF01F03384629460027ADF80430E3
:1072DC008DF806408DF8077006F078FC202001210F
:1072EC0006F034FA39464FF4004006F0FFFC29460C
:1072FC0006488DF806408DF80760ADF8046006F07E
:10730C0065FC3846BDE8FE850008014000140140CC
:10731C00000C0140704700BFFEE700BFFEE700BF56
:10732C00FEE700BFFEE700BF704700BF704700BF1D
:10733C00704700BF704700BF704700BF704700BF69
:10734C00704700BF704700BF704700BF704700BF59
:10735C00704700BF704700BF704700BF704700BF49
:10736C00704700BF704700BF704700BF704700BF39
:10737C00704700BF704700BF704700BF08B5024B95
:10738C001B68984708BD00BF2403002008B5024BBA
:10739C001B68984708BD00BF80040020684620F099
:1073AC000701044B8D4601B51B689847BDE80140A9
:1073BC00854670475404002008B5024B1B6898475B
:1073CC0008BD00BF5C040020704700BF704700BFC1
:1073DC00704700BF704700BF704700BF704700BFC9
:1073EC00704700BF704700BF704700BF704700BFB9
:1073FC00704700BF704700BF704700BF704700BFA9
:10740C00704700BF704700BF704700BF704700BF98
:10741C00704700BF704700BF704700BF704700BF88
:10742C00704700BF704700BF704700BF704700BF78
:10743C00704700BF704700BF704700BF704700BF68
:10744C00684620F007018D4601B5002303E00B4987
:10745C005958995004330A4A0A4998188842F6D365
:10746C00094B02E0002243F8042B084A9342F9D35B
:10747C00FCF7B4FEBDE801408546704720FA0008D1
:10748C00000000207801002078010020180D002059
:10749C00024B33F8100080B2704700BF1C02002072
:1074AC00024B03EB40031982704700BF1C02002003
:1074BC00024B03EB4003188A704700BF1C020020EC
:1074CC0010B50A4C24781CB9002914BF0A461A4678
:1074DC0050214843064B424302991878039B0028DD
:1074EC0008BF0B4692FBF3F010BD00BF4C09002007
:1074FC004E090020044B44F2740202FB00304FF49E
:10750C00805190FBF1F070470060FCFD014B18704E
:10751C00704700BF4E090020014B1870704700BF28
:10752C004C090020074B10B51B68074C34F81300AE
:10753C0080B2FFF7DFFF20220146206A03F0C4FC73
:10754C00206210BD280000201C020020F8B5114B51
:10755C00114E1B68044636F8130080B2FFF7CAFFC1
:10756C000E4B05461B6836F8130080B2FFF7C2FFBE
:10757C00064605FB05F006FB060077197F4207FB64
:10758C00070003F0F9FBA780A060668025802046E9
:10759C00F8BD00BF100200201C02002024000020B7
:1075AC0038B5104C257885B1012D1AD10E4B5B6A7C
:1075BC00002BB8BF5B42B3F5E16F12DDFFF73EFD68
:1075CC0000232370094B1D700BE0074B5B6AC7331C
:1075DC00B3F5C77F05D8FFF729FD044A01231370C3
:1075EC00237038BD4E0900201C0200204D090020DC
:1075FC002DE9F74F534C00250746656252488846E3
:10760C0092469946DDF834B005F000FCC8F5E16807
:10761C00404501D307241EE04C4B626A1B68002ACC
:10762C0034F8130004EB43010B8A80B2B8BF52420A
:10763C00C01A80EAE073A3EBE07393420E9BC8BFC1
:10764C00606251460193CDF800B04A460C9BFFF79F
:10765C0037FF062405463C4805F0DCFB404501D3CA
:10766C00002621E03A4A374B1268596A33F8120067
:10767C0003EB4206328A80B2801A81EAE172A2EBF5
:10768C00E17280EAE071A1EBE0719142C8BF5862EF
:10769C000E9BCDF800B0019351464A460C9BFFF768
:1076AC000FFF24F002040646274805F0B7FB4045BF
:1076BC0002D34FF0000822E0264A224B1268596A86
:1076CC0033F8120003EB420CBCF8102080B2801A85
:1076DC0081EAE172A2EBE17280EAE071A1EBE07168
:1076EC009142C8BF58620E9BCDF800B00193514631
:1076FC004A460C9BFFF7E4FE24F004048046022C5F
:10770C0007D0042C09D0012C0BD108EB06056D42D7
:10771C0007E008EB0506764203E006EB0508C8F126
:10772C00000805FB05F006FB060008FB080003F04B
:10773C0023FBA7F80480B8607E803D803846BDE806
:10774C00FE8F00BF1C020020002C01401002002004
:10775C00240000202800002070B590B0FFF724FD15
:10776C000120014605F0E4FF01214FF4007005F003
:10777C00EDFF414806F0FCFB404B00240093404BCE
:10778C000726019380230593DB18069303F54073BA
:10779C000793A3F5787338486946089303F5FF53AC
:1077AC0009930294039604940A9406F051FC012167
:1077BC00314806F07DFC01254FF4602331480BA9BC
:1077CC000D930B948DF830508DF831400E948DF84C
:1077DC003C6006F0D5FF2C4B2A4819782A46032327
:1077EC0007F050F8294B022219782648032307F09A
:1077FC0049F8274B032219782248134607F042F820
:10780C00244B042219781F48032307F03BF8224B22
:10781C00052219781B48032307F034F81F4B062266
:10782C0019781848032307F02DF81D4B32461978A8
:10783C001448032307F026F8224612484FF4FC6143
:10784C0006F0E2FF0F48294606F0D4FF0D48294602
:10785C0006F0C6FF0B4806F0E1FF0A4806F0E4FF0D
:10786C000028FAD1074806F0E3FF064806F0E6FFC9
:10787C000028FAD110B070BD080002404C24014021
:10788C001C020020002401401C0000201D000020D0
:10789C001E0000201F0000202000002021000020DE
:1078AC0022000020F0B54469856903466543881AB7
:1078BC004FF47A7C002895FBFCF6B8BF4042B042EE
:1078CC00B8BF0CFB00F5104E4FF47A7C30682D18C5
:1078DC0095FBFCF00CFB105737600CB9114611E00E
:1078EC00914205DA1B6841189942A8BF194609E074
:1078FC0008DD064A1B6895FBF2F569185B42994254
:10790C00B8BF19460846F0BD4402002018FCFFFF22
:10791C002DE9F047044690F821000D46062816463E
:10792C009846DDF820A027681ED10868014607F0AC
:10793C00C9FA3E4907F0C6FA814694F8250040087A
:10794C0007F06CFA0146484607F0BCFA63698146B9
:10795C007820584307F062FA0146484607F066FB68
:10796C0007F076FC034611E0072801D000230DE058
:10797C000868014607F0A6FA2D4907F057FB07F0F7
:10798C0067FC236C6269434393FBF2F3C245C8EB7B
:10799C000A08B8BF7F42B8F1000FB8BFC8F10008A1
:1079AC004FF480409845D8BF002701F023F80128F8
:1079BC0003D1304607F032FA31E0384607F02EFAA0
:1079CC002E6880464146304607F01AFC70B1A0691B
:1079DC00636937B90B225043584307F01BFA15491A
:1079EC0017E0584307F016FA134912E041463046A7
:1079FC0007F024FCA0B1A069636937B90B2250438E
:107A0C00584307F007FA0D4903E0584307F002FA10
:107A1C000B4907F00BFB0146304607F04BF9286089
:107A2C00286807F015FCBDE8F08700BF0000C040D7
:107A3C000000F04200401C4600007A4400401CC686
:107A4C0000007AC4024B00229A601A605A60704798
:107A5C004802002070B54668044615460846324672
:107A6C0071421E4603F010FA636B00B2B360736888
:107A7C00A16B451BE818F1603560706011B1104BBB
:107A8C0093FBF1F10A46494203F0FEF90346F06814
:107A9C00B168326858434A434FF4803190FBF1F09F
:107AAC00A1F57F4192FBF1F2801830617360A1F572
:107ABC00014147F6FF7203F0E7F900B270BD00BF59
:107ACC000000FF7F2DE9F04F87B0B04DBDF840406E
:107ADC00BDF842C0AC81A5F80EC00446E8689B46D0
:107AEC00DDF84C808A469146159E02F093FDC0F35A
:107AFC000F43ADF81230ADF81000049BB8F80070CD
:107B0C002B6194F82130062B03D0072B40F01B82FD
:107B1C0010E002F06DF994F8243085B2012B03D1FA
:107B2C0005F5FE45FF35ADB22DB2284602F054F9ED
:107B3C000020F5E102F0D4FA012840F0DE814FF488
:107B4C00007000F057FF012801D1189B5BB94FF46E
:107B5C00006000F04FFF012840F0BE81D8F80030E3
:107B6C00002B00F0B98194F82E00012800F0588108
:107B7C0004D30228854D40F09C8153E0834D42F2A2
:107B8C0010716B6801338B426B6026D8E56BB4F8CF
:107B9C006E205D43B2F5007FB5FBF1F5ADB202D0BE
:107BAC00B2F5806F02D12BB2C8F80030002002F081
:107BBC0013F9002002F0A4FA0021754802F0CEFC63
:107BCC0002A9C0F30F43ADF8080004223046ADF80B
:107BDC000A30002706F0A0FFC7E14FF0000840462E
:107BEC00C5F8048002F084FA94F84630584643F005
:107BFC00010384F84630A5F81680A5F8148000F02F
:107C0C0045FA504600F042FA1699179A00230B6079
:107C1C004046136002F05EFA4FF4004000F0DAFECA
:107C2C004546A2E12B68032B00F2AE80DFE803F09F
:107C3C000241B4B46B6842F210729342DFF84CB15B
:107C4C002AD8E56B01335D43CBF804300020B5FB3B
:107C5C00F2F502F0C1F8002002F052FA00210BF10B
:107C6C00100002F07BFC0422C0F30F43ADF80800B7
:107C7C0002A93046ADF80A3006F04EFFB4F86E306B
:107C8C00ADB2B3F5007F03D0B3F5806F40F0BA808E
:107C9C002BB2C8F80030B5E0002002F029FA94F8B5
:107CAC00463043F0020384F846300123CBF8003011
:107CBC006AE0AD6894F8252085EAE5705208A0EBDF
:107CCC00E570C2EB02418842304B5BDAA16EE7698A
:107CDC00C1EBC1314F435743B4F86E202D48B2F578
:107CEC00007F97FBF0F702D0B2F5806F11D1179A95
:107CFC000021D2F800B0584607F0A0FA08B1ED1BED
:107D0C0005E05846002107F07BFA70B17D191F4B36
:107D1C000AE0B2F5006F08D1D8F80020002A01DD86
:107D2C00ED1B01E001D07D199D60184F0020A58F3F
:107D3C0002F052F8B86802F0E3F9B7F9081007F14D
:107D4C00100002F00BFC0422C0F30F43ADF8080046
:107D5C0002A93046ADF80A3006F0DEFEB4F86E30FB
:107D6C00B3F5007F02D0B3F5806F02D12BB2C8F807
:107D7C00003094F8467017F0020743D1034B0222EF
:107D8C001A6040E003221A6000253CE04802002003
:107D9C0058020020C02709004FF00003AB82EB8291
:107DAC00584600F073F9504600F070F9169900230C
:107DBC002A680B601799022A0B6005D1002002F08B
:107DCC0089F94FF4004000E080207F4D00F002FE66
:107DDC00002002F001F8A86802F092F9B5F9081039
:107DEC0005F1100002F0BAFB0025C0F30F43ADF80B
:107DFC00080002A930460422ADF80A302F4606F0DE
:107E0C008BFE00E00027DFF8C0816420D8F800303A
:107E1C00584300F0CDFDD8F8080000F0CFFDA4E0E9
:107E2C00FFF7ACF9684D01468046287E01F0AAFFA9
:107E3C0085F818801FFA80F801F0DAFF05B22846A1
:107E4C0001F0CAFF18F4004F03D005F5D445AA354C
:107E5C0007E0B8F1000F00F0AF8005F5144505F50B
:107E6C00AA75B4F9400094F8253045435B0895FB9E
:107E7C00F3F04FF6FF7390FBF3F080B202F04CF985
:107E8C0002F05CF9504B4FF00002DA829A82054600
:107E9C00584600F0FBF8504600F0F8F8002002F0CD
:107EAC0019F94FF4004000F095FD05F5004501353A
:107EBC0034E005F11000002102F050FB0027C0F364
:107ECC000F43ADF8080002A930460422ADF80A3081
:107EDC003D4606F021FE48E000213C4802F03EFB06
:107EEC0002A9C0F30F43ADF8080004223046002568
:107EFC00ADF80A3006F010FE36E002F01FF994F8E7
:107F0C002E3000F500450135012BADB203D101F047
:107F1C006FFF00B200E0002001F05EFF2DB228469A
:107F2C0002F0EEF82946294802F018FB02A9C0F32A
:107F3C000F43ADF8080004223046ADF80A30002596
:107F4C0006F0EAFD11E005F11000002102F006FB3D
:107F5C0002A9C0F30F43ADF8080004223046ADF877
:107F6C000A3006F0D9FD00252F4639B25346B6F932
:107F7C0000202046FFF76EFD134F4B46B88229B206
:107F8C00B6F902202046FFF765FDF88207F11400D0
:107F9C0002F040FA07F1140002F062FAC0F30F434A
:107FAC00ADF80000ADF80230009B1846FB6101F003
:107FBC0043FC07B0BDE8F08F01F01AFF00F5FE405E
:107FCC00FF3085B271E700BF480200205802002044
:107FDC0070B50668044615460846324671421E4680
:107FEC0002F052FF636D451BB360A36D1649F3603D
:107FFC00284635604FF6FF7202F046FF0346706864
:10800C00F16818183360706019B163681B0493FB36
:10801C00F1F10A46494202F037FF0346F068B168B5
:10802C00326858434A434FF4803190FBF1F0A1F58C
:10803C007F4192FBF1F280183061736061680A46EF
:10804C00494202F021FF70BD0100FFFF70B5066DC3
:10805C001D4604469E60881A0023EB6028600A497E
:10806C004FF6FF7202F010FF0346A8684FF48072BF
:10807C00584390FBF2F028612B6021680A46494274
:10808C0002F002FF70BD00BF0100FFFF002303617F
:10809C0003604360704700BF094B19685A689142EE
:1080AC0001D100200BE01A68D118097A0132017055
:1080BC001A601A68202A01D100221A600120704728
:1080CC0068020020014B9862704700BF68020020D4
:1080DC00034B1A78104612B100221A700120704717
:1080EC005009002038B50B4B8446DC6A1A6B0134FE
:1080FC00202C08BF002494420AD0DD6A0648ED18F3
:10810C0085F834C040F227710122DC6204F0B8F823
:10811C0038BD00BF680200200048004038B5054655
:10812C00002401E0FFF7DEFF2B5D01341846002B25
:10813C00F8D138BD70B5294C238813F0200F1AD014
:10814C00FFF706F808B1A38815E0254B5A681968A3
:10815C000132202A08BF00228A4205D05968A08823
:10816C00C918C0B208725A601E4B0A221A601C4B06
:10817C009A6A1D4B1A60194E338813F0800F1BD06E
:10818C00194B1C68C4B9164DEA6A2B6B9A420DD078
:10819C00FEF7D2FF2B6B5A1992F834200133B280C0
:1081AC002B632B6B202B07D12C6305E0304622462A
:1081BC0040F2277104F064F80848038813F0400F6C
:1081CC000AD040F2266104F053F9054B1A6BDB6AB6
:1081DC009A4201D1FEF7B6FF70BD00BF00480040C7
:1081EC0068020020540900205809002030B50546CB
:1081FC0087B0544804F08CF94FF48020012105F02D
:10820C00B3FA0820012105F0A1FA0820002105F09D
:10821C00B9FA4D48002105F069FD06AC4FF48063B6
:10822C0024F8043D0323494821468DF816301533B4
:10823C008DF8173005F0CAFC042344488DF817302C
:10824C0021464FF40063ADF8143005F0BFFC6846CE
:10825C0003F0E0FF0B2D25D8DFE805F02406090C10
:10826C000F1215181B1E20224FF461531CE04FF403
:10827C00964319E04FF4E14316E04FF4164313E034
:10828C004FF4614310E04FF496330DE04FF4E133BB
:10829C000AE04FF4613307E02D4B05E02D4B03E072
:1082AC002D4B01E04FF4165369462648009304F019
:1082BC00E7F827230024012504A88DF810300523A6
:1082CC008DF811308DF812408DF8135005F00CFB21
:1082DC001C4840F2FF3104F0A7F828212246194827
:1082EC0003F0CEFF2A46174840F2277103F0C8FF6F
:1082FC002A46144840F2266103F0C2FF2A46114870
:10830C0040F2255103F0BCFF22460E4840F22441B6
:10831C0003F0B6FF22460B4840F6460103F0B0FFCF
:10832C002246084840F66A1103F0AAFF6021224653
:10833C00044803F0A5FF2946024803F093FF07B059
:10834C0030BD00BF0048004010001400000C01407C
:10835C0090D0030020A1070040420F00014B0322E4
:10836C001A607047BC020020044A054B927A0AB18D
:10837C00052200E001221A60704700BF6C09002042
:10838C00BC020020704700BF014B00225A607047AE
:10839C00BC02002008B5074B1A6892B242F00802E2
:1083AC001A601A6892B242F004021A60FFF7D6FF04
:1083BC0008BD00BF405C004010B5064C4FF6FB7387
:1083CC00226802EA03032360FFF7CEFF4FF4064353
:1083DC00236010BD405C0040072818BF1F4B10B530
:1083EC001E4C18BF18702378052B33D8DFE803F028
:1083FC0003060A0E1621FFF7DFFF2BE0FFF7DCFF69
:10840C00042328E002236370013324E06378013BEA
:10841C00DBB263706378FBB9042218E0104B1A6866
:10842C0092B242F010021A6005232370DB186370BD
:10843C0012E06378013BDBB26370637863B9084A7E
:10844C004FF6EF73116801EA030313600622034B26
:10845C001A7001E00623237010BD00BFD009002064
:10846C00405C0040034B9B7A13B1034B05221A600E
:10847C00704700BF6C090020BC020020014B042295
:10848C001A607047BC020020034B1A7A202A01D1D3
:10849C0000221A72704700BFBC020020704700BF58
:1084AC00212808B508D1124B1B681B7803F07F03F9
:1084BC00212B1AD10F4B0EE0202816D10C4B0E4A53
:1084CC001B681B7810720D4A03F07F03212B0CBF25
:1084DC00134600234BB1064A4FF0000112680020EE
:1084EC00518293619847002000E0022008BD00BF34
:1084FC00CC09002041850008BC0200205D850008E5
:10850C00074B1B681B7803F07F03212B05D1022836
:10851C0001D0222801D1002000E00220704700BFCA
:10852C00CC09002019B9012801D8084600E0022026
:10853C00704700BF28B9044B4FF008021B681A8221
:10854C0000E00248704700BFCC0900204400002026
:10855C0028B9044B4FF008021B681A8200E002484D
:10856C00704700BFCC090020440000200B4B10B515
:10857C00DA6882B11B68052B01D000220BE00023C6
:10858C0003E00749595CC15401330449CC68A34248
:10859C00F7D30023CB60104610BD00BFBC020020F7
:1085AC00D8090020084BDB68082B01D800200AE012
:1085BC000023064A9A5CC2540133092BF9D1024BB1
:1085CC000022DA6001207047BC020020D80900208C
:1085DC00704700BF10B5074C0B468AB2C0216360D0
:1085EC0003F082F80120A18802F0AAFE012002F01B
:1085FC0075FD10BDBC02002008B5064B1B68DB786E
:10860C00042B01D9002004E0034901EBC30103F062
:10861C00CBFA08BDCC0900204C00002008B502495B
:10862C0003F0C2FA08BD00BF6C00002008B5024977
:10863C0003F0BAFA08BD00BF74000020334B10B52C
:10864C001B686FF03F0200245A72DC729C72204649
:10865C0002F0BCFC20464FF4007102F0D5FC102156
:10866C00204602F0E7FC4021204602F03DFE80212E
:10867C00204602F029FE204602F066FD244B2046DF
:10868C0093F8641002F07EFE204602F035FD0120C6
:10869C00214602F0B9FC0120C02102F015FE012098
:1086AC00202102F0C7FC0120214602F0DBFC022055
:1086BC004FF4C06102F0A8FC02204FF4807102F06C
:1086CC0003FE0220214602F0CDFC0220202102F004
:1086DC00B1FC0320214602F097FC03204FF4887173
:1086EC0002F002FE0320402102F04CFE03204FF466
:1086FC00405102F0B7FC2146032002F09BFC2046BF
:10870C0003F060FA034B01221A6010BDCC09002063
:10871C0044000020BC02002008B5174B174A19680A
:10872C0089B2118016491288098801EA020212F4F2
:10873C00806F05D04FF6FF321A60124BDB6B9847F7
:10874C000E4B1A880E4B1B8803EA020212F4007FB0
:10875C0008D009490C4A4FF6FF500860117C0131D2
:10876C00C9B21174054A1288134013F4004F01D09A
:10877C0003F026F808BD00BF445C00405E090020F1
:10878C00180A002044000020BC02002010B5032071
:10879C0002F028FE064C034602464FF48871054849
:1087AC00E36002F0B9FF032002F0A6FC10BD00BF8D
:1087BC00BC020020D809002008B5064A064B20B19F
:1087CC001068198805F06AFA03E01068198805F03A
:1087DC0063FA08BD680900206409002038B5064D0D
:1087EC0001232B60054B002420461C60FFF7E4FF9F
:1087FC0003232B60204638BD405C0040445C0040A5
:10880C0008B5FFF7EBFF08BD08B50120FFF7D4FF53
:10881C00064B0121196006494FF4E0520A800549C4
:10882C000020186008601A6008BD00BF405C004062
:10883C00180A0020445C0040084B10B51B6800244B
:10884C009C72FFF7E1FF064A4FF406431460043AAA
:10885C001360044A1460044A138010BDCC09002034
:10886C00445C0040BC020020180A002007B514220A
:10887C0000238DF8042001A801228DF806308DF814
:10888C0007208DF8053005F02FF80EBD002008B537
:10889C0004F0D2FE4FF40000012104F065FF08BD86
:1088AC00F7B5184C184E194F194D9DF820C0316072
:1088BC002A8038600999302204F17E0084F87230E5
:1088CC0084F873C006F028F90A99182204F1B20052
:1088DC0006F022F9FFF7DAFFFFF7C8FF03F034F8D0
:1088EC003868012104F032FF03232D888DF80630FF
:1088FC0030680D3301A9ADF804508DF8073005F040
:10890C0065F9FEBD4400002068090020D409002050
:10891C0064090020014B1868704700BF380A00201A
:10892C00014B1868704700BF300A0020014B1868D3
:10893C00704700BF2C0A0020014B1868704700BF1D
:10894C00280A0020014B1868704700BF340A002029
:10895C00014B1868704700BF1C0A0020014B1868B7
:10896C00704700BF240A0020014B1868704700BFF5
:10897C00200A0020014B1860704700BF380A002005
:10898C00014B1860704700BF300A0020014B186083
:10899C00704700BF2C0A0020014B1860704700BFC5
:1089AC00280A0020014B1860704700BF340A0020D1
:1089BC00014B1860704700BF1C0A0020014B186067
:1089CC00704700BF240A0020014B1860704700BF9D
:1089DC00200A0020024B1A6840EA02021A60704713
:1089EC00D0020020024B1A6822EA00021A6070477B
:1089FC00D0020020034B1B6818420CBF0020012042
:108A0C00704700BFD002002008B56D20FFF7EAFFC9
:108A1C0008BD00BF034B10B51C68FFF7F5FF2046DF
:108A2C0010BD00BFD0020020034B10B51C68FFF72F
:108A3C00EBFF04F06F0010BDD002002062B670474F
:108A4C0072B6704708B5FEF727FB08BD08B5FEF7F0
:108A5C001BFB08BD08B510B104F0E4FF01E004F005
:108A6C00E9FF08BD07B5104B1B78E3B1FEF7FAFA26
:108A7C00FEF71AFBFEF73EFB002301E0019B0133DE
:108A8C000193019A094B9A42F8D9FEF715FBFEF7B0
:108A9C0029FB002301E0019B01330193019A034B55
:108AAC009A42E3D8F7E70EBD810300203F0D030087
:108ABC0008B5FEF795FB014B187008BD810300202B
:108ACC0070B5044600200E4615460321024602F0FE
:108ADC000BF80020C4F30721024602F005F8002031
:108AEC00E1B2024602F000F8002407E0944214BF01
:108AFC000022012201F0F8FF3055013400206A1EDB
:108B0C00AC420146F2D370BD2DE9F04104460F464C
:108B1C00164600200621012201F0E6FF0020052167
:108B2C00024601F0E1FF00200122014601F0DCFFCA
:108B3C0010F0020FF2D000200221024601F0D4FF07
:108B4C000020C4F30721024601F0CEFF0020E1B261
:108B5C00024601F0C9FF002543E0013414F03F0840
:108B6C00795D01D1012204E0721E954214BF0022EE
:108B7C000122002001F0B8FFB8F1000F30D1731EB4
:108B8C009D422DD200200521024601F0ADFF0020B0
:108B9C000122014601F0A8FF10F00100F2D10621DC
:108BAC00012201F0A1FF00200521024601F09CFFEB
:108BBC0000200122014601F097FF10F0020FF2D0C5
:108BCC0000200221024601F08FFF0020C4F3072190
:108BDC00024601F089FF0020E1B2024601F084FF59
:108BEC000135B542B9D300200521024601F07CFFC6
:108BFC0000200122014601F077FF10F0010FF2D1A5
:108C0C00BDE8F08110B5044600200321024601F0B6
:108C1C006BFF0020C4F30721024601F065FF002022
:108C2C00E1B2024601F060FF00200146012201F092
:108C3C005BFF10BD38B5012204460D46002006210D
:108C4C0001F052FF00200521024601F04DFF0020EB
:108C5C000122014601F048FF10F0020FF2D0002073
:108C6C000221024601F040FF0020C4F30721024616
:108C7C0001F03AFF0020E1B2024601F035FF29462F
:108C8C000020012201F030FF00200521024601F0F6
:108C9C002BFF00200122014601F026FF10F0010FEE
:108CAC00F2D138BD38B50725454305F500650C46AE
:108CBC00284609780135FFF7BDFF28466178013554
:108CCC00FFF7B8FF2846A1780135FFF7B3FF284618
:108CDC0021790135FFF7AEFF284661790135FFF7A1
:108CEC00A9FF2846A179FFF7A5FF681CE179FFF7DA
:108CFC00A1FF38BD37B50725454300200C46024679
:108D0C00032101F0F1FE05F500650020C5F30721F4
:108D1C00024601F0E9FE0020E9B2024601F0E4FE51
:108D2C0000200146024601F0DFFE8DF80000002015
:108D3C000146024601F0D8FE8DF8010000200146E4
:108D4C00024601F0D1FE8DF80200002001460246D9
:108D5C0001F0CAFE8DF8040000200146024601F025
:108D6C00C3FE8DF8050000200146024601F0BCFE52
:108D7C008DF8060000200122014601F0B5FE2368A3
:108D8C00009A23F07F4322F07F429A428DF807002D
:108D9C0001D0002005E063680198984214BF0020C0
:108DAC0001203EBD38B5214B1C683BE0002006215C
:108DBC00012201F099FE00200521024601F094FEEB
:108DCC0000200122014601F08FFE10F0020FF2D0BC
:108DDC0000200221024601F087FE0020C4F3072187
:108DEC00024601F081FE0020E1B2024601F07CFE59
:108DFC00002500203F2D14BF002201220146013521
:108E0C0001F072FE402DF4D100200521024601F044
:108E1C006BFE00200122014601F066FE10F0010FEE
:108E2C00F2D14034B4F5804FC0D338BD10000020CF
:108E3C00194B70B5054618680C46FFF7E3FE174B47
:108E4C001B78834202D1164B1B78BBB1124E00210A
:108E5C003068FFF7EFFEFFF7A5FF124B29461868A5
:108E6C002822FFF751FE104B214618687022FFF79D
:108E7C004BFE0A4B30681978FFF7DCFE094B29468C
:108E8C0018682822FFF71CFE074B21461868702231
:108E9C00FFF716FE70BD00BF0C0000200000002084
:108EAC0081030020780100200400002038B507253C
:108EBC00454300200C460246032101F015FE05F542
:108ECC0000650020C5F30721024601F00DFE0020CD
:108EDC00E9B2024601F008FE00200146024601F00C
:108EEC0003FE207000200146024601F0FDFD60707B
:108EFC0000200146024601F0F7FDA070002001465B
:108F0C00024601F0F1FD207100200146024601F0FD
:108F1C00EBFD607100200146024601F0E5FDA071F9
:108F2C0000200146012201F0DFFDE07138BD00BFD9
:108F3C00084B9A7852B95B78142B05D8064A1168FD
:108F4C00064A42F8231004E0032200E00422044BFA
:108F5C001A707047180300207C030020280300209F
:108F6C0074040020054B01205A7805498242087090
:108F7C0002D15A68034B1A60704700BF18030020D7
:108F8C006004002020040020014B02221A7070475C
:108F9C0060040020074A00231360074A1370074A35
:108FAC001360074A1360074A1370074A1360074A95
:108FBC001360704720030020600400202004002070
:108FCC0068040020140300207C030020AC04002063
:108FDC00014B00221A7070476004002030B5234BFF
:108FEC005B78032B3ED8DFE803F008022F39204BC7
:108FFC0018681E4B5C68002322E01D4A1368092B7D
:10900C0007D81A491B484C68591C40F8234011607A
:10901C002BE0092227E052F82350591CA5420ED10F
:10902C0002EB810204E052F8041C013342F8081CE4
:10903C00411E04328B42F6D30D4B196015E00B46E2
:10904C0083420C4AE7D310E0094A00231360094A13
:10905C00002199500433282BF9D106E0064B0A2243
:10906C005A6002E00322044B1A7030BD1803002032
:10907C00640400202404002074040020264A274B9A
:10908C005278092A3BD8DFE802F0050A0F141A229D
:10909C00282E343720491A6849688A182EE01E4A4F
:1090AC00196852688A1A29E01B4A196852684A439F
:1090BC0024E0194A1968526891FBF2F21EE0164A34
:1090CC001968526891FBF2F002FB101216E012497B
:1090DC001A68496801EA020210E00F491A684968E7
:1090EC0041EA02020AE00C491A68496881EA020264
:1090FC0004E01A68D24301E0074A52681A60074A32
:10910C00074B12681AB91A6842F0080202E01A6892
:10911C0022F008021A607047180300207C0300201C
:10912C00200300202A4A2B4B52780A2A43D8DFE826
:10913C0002F0060B11161C242A30363A3D00264943
:10914C001A6809688A1803E0234A196812688A1A8F
:10915C001A6030E0204A196812684A43F8E71E4A40
:10916C001968126891FBF2F2F2E71B4A196812684F
:10917C0091FBF2F002FB1012EAE717491A68096832
:10918C0001EA0202E4E714491A68096841EA02029A
:10919C00DEE711491A68096881EA0202D8E70E4B2A
:1091AC001A68D243D4E71A680B4BD1E70A4A1868FD
:1091BC00116810601960074A084B12681AB91A68CE
:1091CC0042F0080202E01A6822F008021A607047A6
:1091DC00180300207C030020AC0400202003002096
:1091EC00134B5B78052B22D8DFE803F003080D1234
:1091FC00171C104B1A6802F00F0217E00D4B1A687F
:10920C0022F0100212E00B4B1A6822F020020DE043
:10921C00084B1A6822F0400208E0064B1A6822F04C
:10922C00800203E0034B1A6822F480721A607047C4
:10923C001803002020030020124B1A68124B5B68A5
:10924C009A4206DD114B196841F0040121F003012B
:10925C000CE00E4B05D1196821F0060141F001011B
:10926C0004E0196821F0070141F002011960074B75
:10927C001AB91A6842F0080202E01A6822F00802D1
:10928C001A6070477C030020180300202003002084
:10929C0010F0020F0CD111F0100F07D0064B042167
:1092AC005A68064B1970064B1A6004E00A2200E05B
:1092BC000822044B1A707047180300206004002029
:1092CC001003002074040020014B00221A70704718
:1092DC00600400200F4B5B78032B1AD8DFE803F0F7
:1092EC00020413150C4B00E00C4B1A680C4B110AC2
:1092FC0093F800C00B4B18780B4B1A7183F807C00E
:10930C009871597105E0094B00E0094B1A68064B3E
:10931C005A6070471803002010030020200400201E
:10932C006004002014030020740400207C0300203F
:10933C00AC040020014B02221A70704780030020FD
:10934C00024B5A68024B1A60704700BF180300208A
:10935C0020040020294B5B780C2B4ED8DFE803F05F
:10936C00070C11161C21262B30353A3F4400244B98
:10937C001B6813F0080F3BE0214B1B6813F0080F20
:10938C0008E01F4B1B6813F0010F31E01C4B1B68EE
:10939C0013F0010F31D12CE0194B1B6813F0040FA3
:1093AC0026E0174B1B6813F0050F21E0144B1B68CC
:1093BC0013F0020F1CE0124B1B6813F0030F17E0A5
:1093CC000F4B1B6813F0100F12E00D4B1B6813F0C2
:1093DC00200F0DE00A4B1B6813F0400F08E0084B00
:1093EC001B6813F0800F03E0054B1B6813F4807FA0
:1093FC0003D0024B5A68034B1A60704718030020C5
:10940C002003002020040020074970B50B68072BAF
:10941C0009D8064A064816684068064D5C1C45F893
:10942C0023600C60106070BD6804002020040020D4
:10943C001803002000040020054B1A6832B10549BE
:10944C00013A51F822101A60034B1960704700BFA3
:10945C00680400200004002020040020014B00229E
:10946C001A70704760040020084B9A784AB95A78F1
:10947C00142A04D85968064B43F8221004E003223E
:10948C0000E00422034B1A70704700BF1803002041
:10949C002803002074040020114B9A7852B95A7892
:1094AC00104B142A04D8104951F822205A6004E0B9
:1094BC00032201E00B4B04221A700C4B1B786BB18E
:1094CC00084B0B495A680B4B0A601AB91A6842F0E0
:1094DC00080202E01A6822F008021A60704700BF06
:1094EC0018030020740400202803002058040020D6
:1094FC007C0300202003002010B5094B9A7852B948
:10950C005C78142C05D8FAF757FF064B43F8240067
:10951C0004E0032200E00422034B1A7010BD00BFCC
:10952C0018030020280300207404002038B5284BB1
:10953C001B788BB9274A284B5268B2F1FF3F04BF06
:10954C00264A12680A214A431A6000F059F9244B42
:10955C00012218601E4B1A701E4B5C7814B1012C42
:10956C0035D10EE000F04CF91D4B1A681A4B821ADB
:10957C00002A1B68B8BF52429A4224D9144B1C7063
:10958C0025E0FFF747FA10F4804507D0154B10493A
:10959C001A68002022F01002087017E00E4C2368A5
:1095AC008BB100F02DF90E4A23681268821A002A3A
:1095BC00B8BF52429A4206D90A4B05491A680D7037
:1095CC0042F0100202E0084B1A68013A1A6038BDEA
:1095DC001403002018030020B00800207C03002096
:1095EC004C040020200300202004002070B5104DF6
:1095FC00104E2868104C32787368B0F5006F6270AA
:10960C0063600FD83146FFF74DFB31462868FFF7F2
:10961C0071FB20B12B6801332B60652300E007231D
:10962C00237004E007232370044B00221A7070BDD2
:10963C001003002018030020740400206004002094
:10964C0037B5124C657815B1012D1AD10FE0104BBE
:10965C00042201A91868FFF733FA6168019A0D4BCF
:10966C00914202D101225A600EE05D600CE0A378B9
:10967C002A2B06D1064B211D18680422FFF744FA49
:10968C0002E0044B03221A703EBD00BF18030020F9
:10969C0008000020740400202DE9F3411E4B1F4CE0
:1096AC005B681F4A0125B3F5006F1570207027DC2D
:1096BC0011EA050624D118466946FFF7F7FB9DF819
:1096CC0000809DF801709DF802C09DF807009DF880
:1096DC0006109DF805209DF80430267284F8018050
:1096EC00A77084F803C020716171A271E3710B4BF8
:1096FC00E95C1A7A01358A18082D1A72F7D108E03C
:10970C000123064A002199540133082BF9D113780F
:10971C001372BDE8FC8100BF1803002084030020F5
:10972C008003002008B50A4B0A491A6802EA0101B5
:10973C0069B95A6840F2D2439A4208D1064B18686C
:10974C00FFF778FAFFF72EFB0120FFF783F908BD2E
:10975C001803002000FFFF000C00002008B5034B8D
:10976C001A68034B5A60FCF73BF908BD7C030020D8
:10977C001803002008B5034B1A68034B5A60FCF71A
:10978C00E3FD08BD7C03002018030020154B1A785C
:10979C00BAB15968144A013159601168134B01313F
:1097AC001160134A196812780131012A196005D128
:1097BC00104B1A6812B11A68013A1A600022094B50
:1097CC0000E001221A700A4B1A78012A09D10A4BBF
:1097DC00196831B11968013919601B680BB9074B4D
:1097EC001A707047D4020020440900203C09002064
:1097FC004100002058090020540900205009002085
:10980C00014B5868704700BFD402002008B50420F3
:10981C0003F08AFC48F6A04003F096FC012003F00C
:10982C0099FC04480321002204F02CF9012003F0D8
:10983C00A7FC08BD9AC3020043F2B60102B24A4328
:10984C00494903144B434FF0020C991891FBFCF15E
:10985C009A1A82B0002992FBFCF2019004DA002AD9
:10986C002ADB002B6CDC04E0002A56DA002B47DCE8
:10987C0034E003F5E150801A4FF4802190FBF1F0B5
:10988C0000F5617080B200EB6242A1F5003193FBF0
:10989C00F1F192B2511A89B2344BB3F820C02CF4C6
:1098AC00005C4FEA0C4C4FEA1C4CA3F820C0988685
:1098BC001A87998702B0704701F5E150801A4FF46E
:1098CC00802390FBF3F000F56170A3F5003380B2B8
:1098DC0092FBF3F291FBF3F182182EE0C3F5E15009
:1098EC00401880144FF4003200F5617091FBF2F1D6
:1098FC0080B2411A93FBF2F289B28A1892B2CBE78A
:10990C0003F5E150801A801400F561704FF40031BA
:10991C0080B292FBF1F28218B9E701F5E150801A9E
:10992C004FF4802390FBF3F000F56170A3F5003346
:10993C0080B291FBF3F100EB6242411A92B2AAE7BA
:10994C00C3F5E15040184FF4802290FBF2F000F583
:10995C006170A2F5003291FBF2F180B2411A89B22A
:10996C0001EB63439AB297E7E0E3FFFF002C014061
:10997C002DE9F0417D4B8EB01C78012C07D121468E
:10998C00402003F0E3FE21464FF4006002E040F675
:10999C000C00012103F0DAFE08AC754803F062FB01
:1099AC00204602F055FF4FF000038DF82830ADF83B
:1099BC0020304FF06003ADF822304FF4E1632146C4
:1099CC006B48ADF824304FF48073ADF8263002F0BC
:1099DC00E7FD684602F046FF4FF07003ADF800302B
:1099EC004FF00103ADF802304FF00403ADF8043032
:1099FC0040F20553ADF806304FF00203ADF80830D5
:109A0C004FF00803ADF80A304FF48073584869469C
:109A1C00ADF80C304FF40073ADF80E3002F0E2FDEF
:109A2C005348694602F026FE0DAC6946504802F0D8
:109A3C0071FE204604F014F94C4B1978012916D10B
:109A4C004C4804F053F918238DF837300323214682
:109A5C008DF8363048484FF47C53ADF8343004F070
:109A6C00B5F845484FF4285104F022F915E01823B5
:109A7C008DF837300323414821468DF836304FF4AA
:109A8C00E063ADF8343004F0A1F84EF20003214647
:109A9C003B48ADF8343004F099F8354C0821204699
:109AAC0003F010F82046082103F016F82046082190
:109ABC0003F01CF84FF40063ADF810304FF48063E2
:109ACC00ADF812304FF4005301254FF0000620463C
:109ADC0004A9ADF81A304FF48043ADF81C30ADF842
:109AEC001460ADF81650ADF8186002F099FE2046DF
:109AFC00294603F0F3F82A462046294602F0EEFEEA
:109B0C002046294602F0D0FF2946204602F0C8FE26
:109B1C000DF130084FF4A06003F0DCFE404603F07A
:109B2C0025FF1A230BA88DF82C308DF82D508DF8AD
:109B3C002E608DF82F5003F0D7FE192340468DF878
:109B4C0030308DF832608DF833508DF8315003F091
:109B5C00CBFE2046294602F0B1FE4FF46173A3867A
:109B6C002F462387A3870EB0BDE8F0811402002096
:109B7C00002C0140C00016000018014000080140F4
:109B8C00000C0140024B1A6801321A60704700BF8A
:109B9C00400A00200028B8BF404240434B6EC969C0
:109BAC004FF0140C48430CFB03FC154B70B51A68B2
:109BBC0044F620655C6890FBF5F5BCFBF1F0642184
:109BCC000132B0FBF1F02D1982421A605D6016DB98
:109BDC009A680C4C501C90FBF1FC01FB1C01DE68DC
:109BEC0054F822004FF47A7CB5FBFCF5361A761942
:109BFC000020586044F82250DE609960186070BDF7
:109C0C00DC020020440A0020014BD868704700BFDA
:109C1C00DC020020014B1868704700BF400A00208E
:109C2C00014B1860704700BF400A002008B5054B77
:109C3C001B7C012B05D1044B044918680422FEF748
:109C4C0063FF08BDDC0200203C0A0020400A002013
:109C5C0008B5054B042218600449FEF731FF044B8C
:109C6C0001221A7408BD00BF3C0A0020400A0020E3
:109C7C00DC020020014B1868704700BFDC0B002091
:109C8C00014B1860704700BFDC0B002008B5074B78
:109C9C001B78012B09D1064B064918680422FEF7E4
:109CAC0033FFFFF7ADFD044B186008BDF002002038
:109CBC00D80B0020DC0B0020D40B002038B50F4B48
:109CCC001B78012B18D1FFF79BFD0D4C4EF65F2234
:109CDC002368C31A002BB8BF5B4293420CDD094BBF
:109CEC00094A1D6810680135194604221D60FEF7EB
:109CFC000BFFFFF785FD206038BD00BFF002002090
:109D0C00D40B0020DC0B0020D80B002008B5074B2F
:109D1C00042218600649FEF7D3FEFFF771FD054BD0
:109D2C0001221860044B1A7008BD00BFD80B00202C
:109D3C00DC0B0020D40B0020F00200200A2341F29F
:109D4C00883243434243094992B230B59BB2084D25
:109D5C00B1FBF2F4B1FBF3F1296006490C60064942
:109D6C00088006490A80064A138030BD001C4E0E3E
:109D7C00E40B0020E80B0020F60B0020F00B002079
:109D8C00EE0B00200138052822D8DFE800F0071779
:109D9C00030F0B13012916D0022912E0052912D04A
:109DAC0003290EE004290ED001290AE006290AD065
:109DBC00052906E0022906D0042902E0032902D075
:109DCC00062905D101E0012003E04FF6FF7000E009
:109DDC00002000B2704700BF014B1860704700BFF5
:109DEC00F4020020014B1868704700BFF4020020F9
:109DFC00012008B5FDF7C2F90138C0B2052801D918
:109E0C00002002E0024B33F8100000B208BD00BF86
:109E1C0060F3000838B5154CFFF790FF002220685E
:109E2C00022102F05BFD1248002303701148124A14
:109E3C0003701248124D03701248216803701248C7
:109E4C00037013802B704FF448750D8508461380F2
:109E5C00194602F08FFF2068012102F021FD2068D5
:109E6C000221012202F03AFD38BD00BF340000206F
:109E7C00E10B0020F80B0020F20B0020E20B00207D
:109E8C00F50B0020F40B0020E00B00200C4B07B569
:109E9C001B78012B01D11B3304E00A4B1B78012BDF
:109EAC0002D11D338DF80430002301A88DF8073042
:109EBC0003F01AFD044B186803F0D4F80EBD00BF74
:109ECC00380000201502002034000020F0B5694B4A
:109EDC0089B01C780546012C16D12046214603F08A
:109EEC0043FC2146042006AC03F030FC204603F072
:109EFC00B7FE03238DF81A3001338DF81B30214641
:109F0C005D484FF0070335E05C4B1E78012E35D1D0
:109F1C000420314603F028FC594B06AC1F78012F66
:109F2C001AD13946202003F011FC204603F098FE8C
:109F3C0003238DF81A30013321468DF81B3051481C
:109F4C004FF4E043ADF8183003F040FE39464FF4BF
:109F5C00805003F0CBFE11E03146082003F0F6FBF5
:109F6C00204603F07DFE482347488DF81B302146E0
:109F7C004FF4E073ADF8183003F028FE434C03AEF9
:109F8C00206803F06FF8304602F062FC4FF0FF33AC
:109F9C0031462068ADF810304FF00003ADF81230A8
:109FAC0002F0FEFA684602F067FC4FF00003ADF8D1
:109FBC0000304FF00203ADF802304FF00B0369464E
:109FCC002068ADF808304FF00303ADF8043002F010
:109FDC00E5FF01224FF44871206802F0CDFC2068A7
:109FEC0002F09AFC0121206802F086FE40212068D4
:109FFC0002F0D0FC0421206802F0A4FE01212068AC
:10A00C0002F06CFE012D6E4628D11A4B1B78012BE9
:10A01C0001D11B3304E0194B1B78012B02D11D33EA
:10A02C008DF81C30194C01250023022607A88DF849
:10A03C001E308DF81D608DF81F5003F055FC206804
:10A04C0041F65F6102F000FF314620682A4602F0BB
:10A05C0045FC294620682A4602F040FC0B4C0021A6
:10A06C00206802F087FE2068012102F019FC09B07B
:10A07C00F0BD00BF38000020000801401502002090
:10A08C001402002000140140000C01403400002098
:10A09C00014B1880704700BFF60B0020014B186075
:10A0AC00704700BFFC0B002010B504460846FFF7B4
:10A0BC00EFFF2046FFF7F2FF10BD00BF014B1878F1
:10A0CC00704700BFF8020020014B00221A70704745
:10A0DC00F8020020014B1870704700BF740100207B
:10A0EC00014B1878704700BF74010020704700BF07
:10A0FC00024B80B21B689884704700BF3C00002064
:10A10C00014B5860704700BFF8020020014B5868A3
:10A11C00704700BFF802002008B5034B01461868D1
:10A12C0002F028FE08BD00BF3C00002008B5024B21
:10A13C00186802F07BFE08BD3C00002008B5084BF7
:10A14C00186802F073FE074B074A1B68C0EB00400F
:10A15C001288B0FBF3F302FB03F080B208BD00BF22
:10A16C003C000020FC0B0020F60B0020164B07B522
:10A17C001B78012B04D107338DF80430143310E015
:10A18C00124B1B78012B04D116338DF80430063397
:10A19C0007E00F4B1B78012B14D116338DF80430CC
:10A1AC0007338DF8003001A800238DF803308DF8AB
:10A1BC00073003F099FB684603F096FB054B1868D3
:10A1CC0002F050FF0EBD00BF160200204000002020
:10A1DC00170200203C000020F0B5864B8BB01C7899
:10A1EC000746012C0D4618D12046214603F0BCFA37
:10A1FC002146042008AC03F0A9FA204603F030FDF8
:10A20C0048238DF8233021464FF007037A48ADF8E8
:10A21C00203003F0DBFC1C233CE0784B1C78012C39
:10A22C001CD10220214603F09FFA08AE21461020D3
:10A23C0003F08CFA304603F013FD48233146704886
:10A24C008DF823304FF4E073ADF8203003F0BEFCF2
:10A25C0021466C4803F04AFD1D231BE06A4B1C7819
:10A26C00012C19D12146042003F07EFA2146082046
:10A27C0008AC03F06BFA204603F0F2FC48238DF88F
:10A28C00233021464FF4E0736048ADF8203003F0E2
:10A29C009DFC1E238DF824300223002409A88DF880
:10A2AC002530013B8DF827308DF8264003F01CFB40
:10A2BC00574B013F186802F0D5FE03A802F0C8FA0C
:10A2CC00012D18BFADF80E40ADF80C40ADF81240A2
:10A2DC004F4C08BF102303A9206808BFADF80E30FF
:10A2EC00ADF8107002F05CF9012D01D1002200E0F4
:10A2FC00022203211346206802F060FB684602F03C
:10A30C00BBFA434B694618684FF00803ADF80830A8
:10A31C0002F044FE374B1B78012B02D14FF00403A3
:10A32C000CE0364B1B78012B02D14FF0080305E0F3
:10A33C00354B1B78012B03D14FF00C03ADF80030DB
:10A34C00334C6946206802F029FE0121206802F096
:10A35C007BFD01210A46206802F0C0FA20684FF00C
:10A36C0000030121838402F09BFA224B1B78012B02
:10A37C0005D10020022103F0E7FC04230EE01F4B63
:10A38C001B78012B01D1022003E01F4B1878012808
:10A39C0005D1082103F0D8FC4FF4807306930023F9
:10A3AC0008248DF81C3006A801338DF81E308DF86A
:10A3BC001D4003F071FD0F4B1B78012B02D18DF862
:10A3CC0024400AE00D4B1B78012B03D00E4B1B785D
:10A3DC00012B02D116338DF824300023012209A859
:10A3EC008DF826308DF827208DF8253003F07CFA77
:10A3FC000BB0F0BD16020020000801404000002008
:10A40C0000100140000C1A0017020020000C014043
:10A41C003C000020B0F90030B0F9022003FB03F13E
:10A42C0002FB021110B50C4CA14214D94FEA116C6D
:10A43C00ACF13A0C09495FFA8CFC31F81CC04FF4B2
:10A44C00004102FB0CF203FB0CF392FBF1F293FBC9
:10A45C00F1F14280018010BD0044FA3A6CF300081F
:10A46C00124B37B5B3F902C0B3F90010B0F90220A2
:10A47C00B0F9000002FB0CF400FB01F500FB0CFC36
:10A48C004A434FF4004395FBF3F194FBF3F492FB36
:10A49C00F3F264189CFBF3F3D31A0020A2B262F31C
:10A4AC000F009BB263F31F403EBD00BF00030020B2
:10A4BC00A0F50040C0F3891000F44073B3F5807F21
:10A4CC0082B037D001DC23B305E0B3F5007F05D0B3
:10A4DC00B3F5407F0FD00023184639E0C0B21E4BB5
:10A4EC00420082F4FF7203EB4000D218B0F88C00EB
:10A4FC00B2F88C302CE0184AC0B202EB400340009A
:10A50C0080F4FF70B3F88C3082185B42B2F88C0088
:10A51C000EE0114BC0B2420082F4FF7203EB40001C
:10A52C00D218B0F88C00B2F88C3040425B4280B24A
:10A53C009BB20DE0C0B2084B420082F4FF72D218FD
:10A54C00B2F88C2003EB40035242B3F88C3090B23B
:10A55C0043EA004002B070476CF3000830B5044683
:10A56C0085B00846FFF7A4FFC0F30F43ADF80230E7
:10A57C00ADF80000134A00994FF400431160B4F990
:10A58C000210B2F90200B4F900C0B2F9002001FBCC
:10A59C0000F50CFB02F40CFB00F04A4394FBF3F4C3
:10A5AC0095FBF3F192FBF3F2641A90FBF3F3D318DF
:10A5BC000020A2B262F30F009BB263F31F4005B000
:10A5CC0030BD00BF00030020032903D8DFE801F0F1
:10A5DC0004081014002018E00D4B03EB400004E0BD
:10A5EC0040000B4B80F4FF70C018B0F88C000CE0EE
:10A5FC00074B03EB400004E04000054B80F4FF7078
:10A60C00C018B0F88C00404280B200B2704700BF56
:10A61C006CF3000883B244F6E61100140FFA83FCC5
:10A62C00484301FB0CF14FF4004291FBF2F190FB1B
:10A63C00F2F290B24A42A2EB4002002063F30F0008
:10A64C0092B284B062F31F4004B0704730B50C4B2B
:10A65C000C4C844622681B689A4201D100200EE003
:10A66C002368094A5D1C02EB03130FCB8CE80F0027
:10A67C0025602368082B01D100232360012030BD05
:10A68C008C0C0020000C00200C0C0020704700BF2C
:10A69C007FB52B4B2B4A19681268914204D10120CB
:10A6AC00002103F057FE48E01968274A02EB01111C
:10A6BC00487850B11B6802EB0312536804228DF8E2
:10A6CC000C2000220192029307E01B68029002EB1F
:10A6DC00031253688DF80C000193194B1A681A4B2E
:10A6EC0003EB02139B781BB102238DF80D3001E0B4
:10A6FC008DF80D30124B00221968134B0901CB5CFD
:10A70C008DF80E300E4B0DF1180C18680CEB020185
:10A71C0002EB001C0C4801326044007A082A01F854
:10A72C00090CEFD11A6801321A601A68082A01D193
:10A73C0000221A6001A803F01BFE07B000BD00BF89
:10A74C00080C0020040C0020900C0020F0B543787D
:10A75C0087B00646426833B104238DF80C300023D1
:10A76C000292019303E0029301928DF80C30B378BE
:10A77C0003B102238DF80D30327800238DF80E20B2
:10A78C00F21801A8117AC2180133082BD172F7D133
:10A79C0003F0EEFD042818D10D4D0E4B2C681B68F0
:10A7AC000134082C08BF00249C4201D100200DE08C
:10A7BC0096E80F002F68084E06EB071C8CE80F007C
:10A7CC00012001462C6003F0C5FD012007B0F0BD4F
:10A7DC00040C0020080C0020900C002030B5294DF2
:10A7EC00294B2C681B680134082C08BF00249C42A0
:10A7FC0087B043D001A903F097FE9DF80C20234BA2
:10A80C00042A09D12A68012103EB021251702A682B
:10A81C0003EB0213029A08E02A68002103EB0212F0
:10A82C0051702A6803EB0213019A5A609DF80D309F
:10A83C00144A022B154B04D1126803EB02130122AC
:10A84C0003E0126803EB021300229A700D4B9DF883
:10A85C000E101A680D4B1201D1540023094A06A997
:10A86C00C8181168094D03EB011110F8090C0133DC
:10A87C004919082B0872F1D1146001E003F038FE7D
:10A88C0007B030BD8C0C0020000C00200C0C0020FC
:10A89C0008B50120FFF7A2FF08BD00BF08B50020D6
:10A8AC00FFF79CFF08BD00BF2DE9F0470C238AB0D1
:10A8BC008DF81C3003238DF81D30013800238DF8E2
:10A8CC001B300C46154607281AD8DFE800F0161383
:10A8DC00100D0A1907044FF0020313E04FF00403A4
:10A8EC0010E04FF010030DE04FF014030AE04FF0AE
:10A8FC00280307E04FF0640304E04FF0C80301E0C5
:10A90C004FF00803ADF81E3003F02EFF4FF000702F
:10A91C00012102F029FF0120014602F017FF04205B
:10A92C00012102F013FF0420002102F02BFF4FF451
:10A93C00EA10002103F0DAF90AAE4FF4805326F83E
:10A94C00043D0323314667488DF8263015338DF8C6
:10A95C00273003F03BF90423314662488DF8273049
:10A96C004FF4006300260127ADF824301FFA84F859
:10A97C0003F02CF905A80DF1040A8DF81A608DF876
:10A98C0014608DF815708DF816608DF817608DF8C1
:10A99C0018708DF8197003F0DBFB4FEA4813ADF813
:10A9AC00083050464FF0FF338DF804608DF8056089
:10A9BC008DF80670ADF80A60ADF80C30ADF80E30BD
:10A9CC00ADF810608DF81270B14603F033FCBDB1D8
:10A9DC006B01ADF8083050464FF0FF338DF8056031
:10A9EC00ADF80A608DF812708DF804708DF8067051
:10A9FC00ADF80C30ADF80E30ADF8107003F01AFC59
:10AA0C004FEAC80343F004030DF1040800270126A4
:10AA1C0002226413ADF80A3040464FF0FF338DF834
:10AA2C000420ADF808408DF805708DF80660ADF87F
:10AA3C000C30ADF80E30ADF810708DF8126003F0DC
:10AA4C00F9FBBD421BDDEB0043F004036D13032245
:10AA5C00ADF80A3040464FF0FF338DF804208DF8E6
:10AA6C000570ADF808508DF812608DF80660ADF8E1
:10AA7C000C30ADF80E30ADF8106003F0DBFB08AF16
:10AA8C00012407260025142338468DF820308DF834
:10AA9C0021608DF822508DF8234002F025FF1523FC
:10AAAC0038468DF820308DF821608DF822508DF8C5
:10AABC00234002F019FF132338468DF820308DF80F
:10AACC0021608DF822508DF8234002F00DFF0220FA
:10AADC00214603F03FFC2146102003F03BFC0AB05A
:10AAEC00BDE8F08700080140F0B5484B87B01B78F3
:10AAFC00044683420D46174644D0454B1B78012B28
:10AB0C0003D1012801D1434E00E0434E00213046D1
:10AB1C0002F094FB4FF00003ADF804304FF4827355
:10AB2C00ADF806304FF00003ADF808304FF00203DB
:10AB3C00ADF80A304FF00103ADF80C304FF4007350
:10AB4C00ADF80E30012C4FF00003ADF81230ADF81B
:10AB5C00143006D002D3022C06D102E04FF01003C1
:10AB6C0004E04FF0080301E04FF0180301A9304650
:10AB7C00ADF8103002F026FB3046012102F05EFBEE
:10AB8C00224B1C70032C3ED8DFE804F00205080BA6
:10AB9C00FCF740FA07E0FCF759FA04E0FCF75AFA24
:10ABAC0001E0FCF75BFA1A4B1B78012B03D1012C4B
:10ABBC0001D1184E00E0184E3046022102F0D2FBB3
:10ABCC000028F9D02946304602F070FB30460121AE
:10ABDC0002F0C8FB0028F9D087B1032C13D8DFE8AA
:10ABEC0004F00205080BFCF71BFA07E0FCF730FA3F
:10ABFC0004E0FCF731FA01E0FCF732FA304602F0DF
:10AC0C0057FBC0B200E0002007B0F0BD04030020E9
:10AC1C001802002000380040003001402DE9F041BE
:10AC2C00012186B04FF4805002F090FD01200146C6
:10AC3C0005AF02F08BFD182403264FF0A003484803
:10AC4C003946ADF814308DF816608DF8174002F0C7
:10AC5C00BDFF4FF0400342483946ADF814308DF833
:10AC6C0016608DF8174002F0B1FF0120002103F0AF
:10AC7C003DF84FF00003ADF800304FF48273ADF89F
:10AC8C0002304FF00003ADF804304FF00203ADF882
:10AC9C0006304FF00103ADF808304FF40073314823
:10ACAC006946ADF80A304FF00003ADF80E30ADF840
:10ACBC001030ADF80C4002F085FA0121294802F061
:10ACCC00BDFA294BE8461D78012D42D14FF4804046
:10ACDC00294602F049FD4AF2000324483946ADF8F2
:10ACEC0014308DF816608DF8174002F06FFF4FF49A
:10ACFC00804339461D48ADF814308DF816608DF838
:10AD0C00174002F063FF4FF00003ADF800304FF432
:10AD1C008273ADF802304FF00003ADF804304FF001
:10AD2C000203ADF806304FF4007369461048ADF8D5
:10AD3C000A304FF00003ADF80C40ADF80850ADF8F8
:10AD4C000E30ADF8103002F03DFA2946084802F0FA
:10AD5C0075FA084B4FF0FF321A7006B0BDE8F0815F
:10AD6C00000801400030014018020020000C014096
:10AD7C00003800400403002003464FF6FF70834266
:10AD8C004EDDB3F1807F27DBB3F1805F11DBB3F1D4
:10AD9C00804F08DB3A4A934270DC3A4A191652F853
:10ADAC002120120212E0374A991552F82120D201C3
:10ADBC000CE0B3F1806F334A04DB191552F82120F3
:10ADCC00920103E0991452F82120520193FBF2F105
:10ADDC000132521852101DE0B3F5801F0DDBB3F594
:10ADEC00800F284A04DB191452F82120120111E0BB
:10ADFC00991352F82120D2000CE0B3F5802F214A90
:10AE0C0004DB191352F82120920003E0991252F836
:10AE1C002120520093FBF2F1501C401840101FE00F
:10AE2C00FF2B23DDB3F5805F0CDBB3F5804F154AA8
:10AE3C0003DB191252F8210011E0991152F821008C
:10AE4C0040100CE0B3F5806F0E4A04DB191152F878
:10AE5C002100801003E0991052F82100C01001303D
:10AE6C0000FB00F29A4209DD013807E0002BA9BF74
:10AE7C00044A4FF0FF3052F823000011704700BF16
:10AE8C000080FE7FF8F50008904203DC8142ACBFE5
:10AE9C000A4602461046704770B5044610460E46E8
:10AEAC0003F0BCFF05462946204604F0C7F940B91B
:10AEBC00304603F0B3FF05462946204604F0A0F9BE
:10AECC0000B12C46204670BD70B514460E4603F0FA
:10AEDC00A5FF0546204603F09DFF04462146284663
:10AEEC0004F0A4F80146284603F0E2FE054630467D
:10AEFC0003F094FF214604F099F80146284603F02C
:10AF0C00D9FE04F0A5F970BD70B51BB12D2301F865
:10AF1C00013B40424B1CB0FBF2F402FB140C5D1ED7
:10AF2C00BCF1090F8CBF0CF1570C0CF1300C03F871
:10AF3C0001CC1E4620460133002CECD134702B780A
:10AF4C000A7805F8012901F8013BA942F7D33046EC
:10AF5C0070BD00BF0A2A08B5844613468E4603D13D
:10AF6C00002801DA012303E01A46604671460023EB
:10AF7C00FFF7CAFF08BD00BF014B1860704700BF48
:10AF8C00405C0040014B186880B27047405C004048
:10AF9C00014B1860704700BF445C0040014B1868BF
:10AFAC0080B27047445C0040014B186880B2704717
:10AFBC00485C0040014B1860704700BF4C5C00407F
:10AFCC00014B186880B270474C5C00404FF6F87328
:10AFDC00024A00EA03031360704700BF505C004054
:10AFEC00014B186880B27047505C0040014B43F82D
:10AFFC0020107047005C0040024B53F8200080B2D8
:10B00C00704700BF005C0040054B10B553F8204062
:10B01C0048F68F1204EA02020A4343F8202010BDBE
:10B02C00005C0040024B53F8200000F4C0607047F5
:10B03C00005C00400A4B10B553F8202048F6BF7452
:10B04C0002EA040411F0100F18BF84F0100411F080
:10B05C00200F18BF84F0200443F8204010BD00BF1F
:10B06C00005C00400A4B10B553F820204BF68F744F
:10B07C0002EA040411F4805F18BF84F4805411F4C4
:10B08C00005F18BF84F4005443F8204010BD00BF8B
:10B09C00005C004038B50D460446FFF7ADFF012DAE
:10B0AC0002D120F4805003E0022D04D120F01000D6
:10B0BC00014B43F8240038BD005C0040024B53F8B0
:10B0CC00200000F030007047005C0040024B53F849
:10B0DC00200000F440507047005C0040054B48F6DF
:10B0EC00BF7253F8201001EA020282F0300243F8DA
:10B0FC0020207047005C0040054B4BF68F7253F8D4
:10B10C00201001EA020282F4405243F820207047DA
:10B11C00005C0040054B48F68F6253F8201001EAA2
:10B12C00020242F4807243F820207047005C004019
:10B13C00044B48F68F6253F8201001EA020243F8E0
:10B14C0020207047005C0040044B48F68F6253F897
:10B15C00201001EA020243F820207047005C0040F6
:10B16C00054B48F68F6253F8201001EA020242F4B4
:10B17C00807243F820207047005C0040054B48F675
:10B18C008F6253F8201001EA020242F4807243F8F5
:10B19C0020207047005C0040044B48F68F6253F847
:10B1AC00201001EA020243F820207047005C0040A6
:10B1BC00044B53F8200000F03000102814BF00207E
:10B1CC0001207047005C0040054B53F8200000F450
:10B1DC004050B0F5805F14BF00200120704700BFC5
:10B1EC00005C0040044B40F68F7253F8201001EACB
:10B1FC00020243F820207047005C0040044B48F6E4
:10B20C000F7253F8201001EA020243F82020704715
:10B21C00005C0040054B48F68F7253F8201001EA91
:10B22C00020242F4804243F820207047005C004048
:10B23C00054B48F68F7253F8201001EA020242F0D7
:10B24C00400243F820207047005C0040084B53F844
:10B25C00202012F4804F09D053F8201048F68F723A
:10B26C0001EA020242F4804243F82020704700BFFA
:10B27C00005C0040084B53F8202012F0400F09D01E
:10B28C0053F8201048F68F7201EA020242F0400295
:10B29C0043F82020704700BF005C0040054B10B500
:10B2AC0053F8204048F68F7204EA02020A4343F82E
:10B2BC00202010BD005C0040024B53F8200000F031
:10B2CC000F007047005C0040064B49081B684900A2
:10B2DC009BB203EBC00303F1005303F540535B0037
:10B2EC0019607047505C0040054A064B12684908CB
:10B2FC0092B202EBC002D3185B0049001960704790
:10B30C00505C004004300020054B1B689BB203EBE3
:10B31C00C00303F1005303F540535B0018887047DA
:10B32C00505C0040044A054B126892B202EBC0021A
:10B33C00D3185B0018887047505C00400430002024
:10B34C00044A054B126892B202EBC002D3185B00A0
:10B35C0019607047505C0040023000203E2909D92A
:10B36C004B0911F01F0F01D1013B9BB29B0243F41F
:10B37C00004305E04B0811F0010F18BF01339B028D
:10B38C00036070470D4A0E4B126892B2D31803EB50
:10B39C00C0035B003E2909D94A0911F01F0F01D1E6
:10B3AC00013A92B2920242F4004205E04A0811F0CE
:10B3BC00010F18BF013292021A607047505C0040B6
:10B3CC0006300020054A064B126892B202EBC0020E
:10B3DC00D3185B0018688005800D7047505C0040E6
:10B3EC0002300020054A064B126892B202EBC002F2
:10B3FC00D3185B0018688005800D7047505C0040C6
:10B40C00063000200C4B30B51D681C68C0001FFABC
:10B41C0085FC8444A4B2094B00190CF1005CC318E0
:10B42C000CF5405C490852084FEA4C0049005B009F
:10B43C00520001601A6030BD505C004004300020A6
:10B44C00064B49081B6849009BB203EBC00303F190
:10B45C00005303F540535B0019607047505C00408B
:10B46C00054A064B1268490892B202EBC002D31887
:10B47C005B00490019607047505C004004300020AC
:10B48C00054B1B689BB203EBC00303F1005303F5A0
:10B49C0040535B0018887047505C0040044A054BD1
:10B4AC00126892B202EBC002D3185B001888704786
:10B4BC00505C004004300020012910B524D1254BEC
:10B4CC0025491B68C0009BB2591809184B003E2A2D
:10B4DC0009D9510912F01F0F01D1013989B2890222
:10B4EC0041F4004105E0510812F0010F18BF013181
:10B4FC00890219601749194B096889B2CB181818B9
:10B50C0040003E2A1ED913E0022922D1114BC00063
:10B51C001C681B68A4B21FFA83FC0F490F4B8444B0
:10B52C0000194118634449005B000A601A6010E07E
:10B53C00530912F01F0F01D1013B9BB29B0243F444
:10B54C00004305E0530812F0010F18BF01339B02B2
:10B55C00036010BD505C004002300020063000201B
:10B56C0001291BD11349144B096889B2CB1803EB81
:10B57C00C00040003E2A09D9530912F01F0F01D117
:10B58C00013B9BB29B0243F4004305E0530812F0CD
:10B59C00010F18BF01339B0203600AE0022908D196
:10B5AC000449054B096889B201EBC000C3185B0064
:10B5BC001A607047505C00400230002001291BD1FA
:10B5CC001349144B096889B2CB1803EBC000400037
:10B5DC003E2A09D9530912F01F0F01D1013B9BB22E
:10B5EC009B0243F4004305E0530812F0010F18BF0F
:10B5FC0001339B0203600AE0022908D10449054B80
:10B60C00096889B201EBC000C3185B001A6070476F
:10B61C00505C004006300020054A064B126892B27E
:10B62C0002EBC002D3185B0018688005800D7047D0
:10B63C00505C004002300020054A064B126892B262
:10B64C0002EBC002D3185B0018688005800D7047B0
:10B65C00505C0040063000200D4BC00019680D4AAC
:10B66C0089B241188A185200128812F47C4F01D00A
:10B67C0001200CE01A68084B92B28018C3185B00CA
:10B68C0018888005800D002814BF02200020704708
:10B69C00505C00400630002002300020012909D106
:10B6AC000B4A48F68F7352F8201001EA030343F05B
:10B6BC0040030AE002290AD1054A48F68F7352F872
:10B6CC00201001EA030343F4804342F82030704712
:10B6DC00005C004041EA0020704700BF030AC0B282
:10B6EC0043EA0020704700BF01F10051013201F51F
:10B6FC00405110B549005208002308E010F803C06F
:10B70C006478013A4CEA042C21F813C00233C418B3
:10B71C00002AF3D110BD00BF01F10051013201F537
:10B72C00405110B549005208002304E031F8134091
:10B73C00013AC4520233002AF8D110BD08B529E0F1
:10B74C0047F6FF700860198801F00F018B0003F1B8
:10B75C008043117003F5B843196889B211F4004F96
:10B76C0009D0186840F68F7100EA0101196012784F
:10B77C000E4B013A0BE011F0800F0BD0186848F615
:10B78C000F7100EA010119601278094B013A53F864
:10B79C00223098470749084B0868084A80B218803D
:10B7AC00188800B20028CBDB08BD00BF2C0100209C
:10B7BC0010010020445C00405E0900206609002056
:10B7CC00F8B59AE047F6FF761E601688564F06F0DD
:10B7DC000F06B30003F1804303F5B8433E70002E0F
:10B7EC0064D127682668236807F4405C03EA0000EC
:10B7FC0080F400502060236806F0300003EA010159
:10B80C0081F0200121601388484A13F0100F10803A
:10B81C00A5F800C004D023689BB213F0800F08D0A9
:10B82C00226848F60F7302EA0303236000F0CEFA95
:10B83C0016E013F4006F08D0226840F68F7302EA0A
:10B84C000303236000F062FB0AE013F4004F54D0B2
:10B85C00226840F68F7302EA0303236000F0F8F9C4
:10B86C0021682A884BF68F7301EA030312F4805F78
:10B87C0018BF83F4805312F4005F2D4A18BF83F471
:10B88C0000531360294B11681A8848F6BF7301EAFC
:10B89C00030312F0100F18BF83F0100312F0200FE7
:10B8AC00234A18BF83F0200313603BE01C68A4B24A
:10B8BC0014F4004F0BD0196840F68F7201EA0202A3
:10B8CC001A603A781B4B013A53F82230984714F01F
:10B8DC00800F12D0144948F60F720B789B0003F1BD
:10B8EC00804303F5B843186800EA02021A600A782C
:10B8FC00114B013A53F822309847104B104A1D68EF
:10B90C000B4C1FFA85FCA2F800C0B2F800C04BF635
:10B91C008F700FFA8CFCBCF1000F48F6BF71094D0B
:10B92C00FFF650AFF8BD00BF66090020120D0020D5
:10B93C00005C00402C01002010010020445C004001
:10B94C005E090020100D0020074A022108B50748A7
:10B95C0011720749074B086007490A60074A1360D0
:10B96C001B68984708BD00BF6C0900204C010020E3
:10B97C00880900207C000020CC09002060090020F0
:10B98C0010B5074C20B922684FF00103138205E073
:10B99C00044B1B681B68984720680A3010BD00BF19
:10B9AC00CC0900208809002010B50A4B0A4A1B68F4
:10B9BC005178DA7891420AD3997841B99C8834B994
:10B9CC009A72064B1B685B689847204600E0022081
:10B9DC0010BD00BFCC0900204801002088090020C0
:10B9EC0010B5074C20B922684FF00103138205E013
:10B9FC00044B1B689B68984720680C3010BD00BF37
:10BA0C00CC0900208809002038B50E4C0E4B22685A
:10BA1C001B68D1789B695079984723689A7A7AB1D8
:10BA2C0070B91A7962B99D7855B9084B1B68DB68F7
:10BA3C009847236828465979DA78D9721A7300E046
:10BA4C00022038BDCC0900206009002088090020A4
:10BA5C0008B50246244B20B91B684FF0020119822D
:10BA6C0040E0224A4FF000011B681180197811F058
:10BA7C007F0113D15B7A13F0200F03D0117841F0C2
:10BA8C000201117013F0400F184B15BF1A781A7879
:10BA9C0022F0010242F001021A701EE0012921D0AD
:10BAAC00022901D000221DE0597911F0800F01F01C
:10BABC000F0306D00E4951F8233003F03003102B3E
:10BACC0006E00B4951F8233003F44053B3F5805F83
:10BADC0003D1137843F001031370064B1B681B69E9
:10BAEC009847024A104608BDCC090020140D0020CE
:10BAFC00005C00408809002010B51E4B19684A797B
:10BB0C0012F0800F22F0800305D01B4850F8230060
:10BB1C0000F0300004E0184850F8230000F44050C6
:10BB2C00164C94F800C0634522D24C8804BBF8B183
:10BB3C00897AE9B112F0800F09D00F4948F6BF722B
:10BB4C0051F8230000EA020282F0100208E00A49D0
:10BB5C004BF68F7251F8230000EA020282F48052F5
:10BB6C0041F82320064B1B689B699847002000E096
:10BB7C00022010BDCC090020005C004048010020D0
:10BB8C008809002008B5064B1B685A7A42F020023F
:10BB9C005A72044B1B68DB699847002008BD00BF34
:10BBAC00CC09002088090020054B1A68538A18B963
:10BBBC008988CB1A138201E008681818704700BFF7
:10BBCC00CC09002030B50E4B1C78002310E05FFA36
:10BBDC0083FC4FEA8C0202F1804202F5B8421568F0
:10BBEC0048F68F7105EA010141EA0C01116001333D
:10BBFC00A342ECD3034B40F08000186030BD00BF73
:10BC0C00480100204C5C0040704700BF08B50C4B4D
:10BC1C00002093F82C10FFF7B5FB0A4B1B68187A21
:10BC2C00082807D1084B4FF480521A80074B4FF06D
:10BC3C0010021A80092814BF0020012008BD00BF83
:10BC4C007C000020CC090020100D0020120D0020DB
:10BC5C0070B52D4B1C68237A032B01D0052B46D1D4
:10BC6C00A369228AABB1A2B1A58A954228BF154619
:10BC7C0028469847228A638A521BEB180646228272
:10BC8C0063820020FFF74EFB2A4601463046FFF741
:10BC9C0043FD238A5BB11D4B4FF4405200201A80A8
:10BCAC000146FFF74DFB1A4B4FF030021A80A28A67
:10BCBC00238A9A4203D8144B03221B6803E0124ACE
:10BCCC001BB1136805221A720DE01268062111725D
:10BCDC00104A1168104A89B28A18520013600C4B32
:10BCEC004FF030021A80084B1B681B7A06E0072BBA
:10BCFC0003D10A4B1B68DB6898470823024A126879
:10BD0C001372FFF783FF70BDCC090020100D0020CB
:10BD1C00120D0020505C0040023000206009002011
:10BD2C00F8B5244B1C68238A267ABBB9042E15D18E
:10BD3C00214822490278012A0BD1214C214A24683E
:10BD4C000370A0B28218520013604FF030020A80C8
:10BD5C002BE04FF010030B80072626E0A68AA26981
:10BD6C009E4234BF35461D462846B34294BF042636
:10BD7C000226904707460020FFF7C6FA2A460146DE
:10BD8C003846FFF7B1FC29460020FFF7D9FA638A41
:10BD9C00228AEB186382094B551B4FF03002258227
:10BDAC001A80094B4FF440521A80024B1B681E72CA
:10BDBC00F8BD00BFCC09002005030020120D0020A7
:10BDCC00505C004002300020100D002008B5144BD0
:10BDDC001B681A7A022A01D0042A05D1FFF7A0FFAA
:10BDEC000F4B1B681B7A14E0062A11D15A78052ACE
:10BDFC000AD11A7812F07F0F06D1D878FFF7E2FE3D
:10BE0C00084B1B681B6A9847074B1B689B68984735
:10BE1C000823034A12681372FFF7F8FE08BD00BF2F
:10BE2C00CC090020880900206009002038B5324B6D
:10BE3C001B68187810F07F0004D15A7A22F0200287
:10BE4C005A7258E0022855D15A88002A52D11A79D0
:10BE5C00002A4FD15A7912F0800F22F0800405D0BD
:10BE6C00264951F8241001F0300104E0234951F81F
:10BE7C00241001F440512248007884423AD200291F
:10BE8C0038D09B7A002B35D012F0800F0FD01B4B83
:10BE9C0053F8243003F03003102B25D1E4B22046A4
:10BEAC00FFF7E8F920463021FFF7C4F81CE0134DEA
:10BEBC0055F8243003F44053B3F5805F14D134B9F2
:10BECC00104B204693F82C10FFF75CFA02E020464A
:10BEDC00FFF7BCF955F824204BF68F7302EA0303E5
:10BEEC0083F4405345F82430074B1B685B69984733
:10BEFC00002000E0022038BDCC090020005C00408E
:10BF0C00480100207C00002088090020F7B58D4BEB
:10BF1C008D4E1A6835688D4B92B2D3182A7A5B0015
:10BF2C00092A1B681BD09BB203F1005303F5405345
:10BF3C005B001C4614F8012B03F10A072A705B788E
:10BF4C006B70B4F80300FFF7C9FB6880B4F8070006
:10BF5C003468FFF7C3FBA08033687F88DF807A4C9E
:10BF6C0001212368DA8819725D78002A62D11A7867
:10BF7C0012F07F022ED1092D02D1FFF715FD3BE007
:10BF8C00052D0DD193F90320002A4EDB9A78002A57
:10BF9C004BD19A88002A48D19B7A002B37D044E0A9
:10BFAC00032D0BD1DA78012A27D19A882ABB5B7A28
:10BFBC0013F0200F21D0FFF7E5FD1DE0012D1CD162
:10BFCC00DA78012A19D19A88BAB95B7A13F0200F62
:10BFDC0013D00AE0012A04D10B2D0ED1FFF714FD6A
:10BFEC000AE0022A09D1012D02D1FFF71FFF03E05D
:10BFFC00032D02D1FFF780FD48B1554B28461B6835
:10C00C005B699847032801D109230FE068B94D4AB1
:10C01C00504B12684FF0300192B2D3185B000022E3
:10C02C001A604D4B1980062300E00823464A12681B
:10C03C001372E3E0062D18D11A7812F07F0F40F03E
:10C04C0097809B78012B03D1414B1B68DB696EE019
:10C05C00022B03D13E4B1B681B6A68E0032B40F09C
:10C06C0087803B4B1B685B6A61E0002D3CD1598893
:10C07C0000297DD15A6822F47F42B2F5003F77D176
:10C08C001A7812F07F0203D19B88002B70D129E023
:10C09C00012A0BD158792E4B1B689B6998470028B5
:10C0AC0066D123689B7A002B62D01BE0022A5FD1F9
:10C0BC005B7913F0800F03F00F0205D0274951F87C
:10C0CC00221001F0300104E0244951F8221001F44F
:10C0DC0040512348007882424AD213F0700F47D166
:10C0EC00002945D01F4B23E0082D05D11B7813F0F8
:10C0FC007F0F3DD11C4B1BE00A2D39D11A7802F071
:10C10C007F02012A34D19A7A002A31D05988002929
:10C11C002ED15A6822F47F42B2F5803F28D158794B
:10C12C000B4B1B689B69984710BB104B00E0FBB195
:10C13C00054A4FF000011268002093615182984724
:10C14C00002020E0505C0040CC090020043000208E
:10C15C006009002002300020120D0020005C00401D
:10C16C00480100205DBA00088DB90008EDB900083F
:10C17C00244C254B22681B6850781B699847032870
:10C18C0001D1236806E01F4B4FF6FF711B681A8A1A
:10C19C008A4201D1092203E0022800D012B90822F8
:10C1AC001A722BE093F90010002921DAD988019139
:10C1BC000198824202D9019A1A8211E08A420FD266
:10C1CC001149096891F82C108A4201D2002105E02E
:10C1DC0092FBF1F001FB102212B901210B4A1170F4
:10C1EC00094A126892F82C209A82FFF799FD05E013
:10C1FC0003221A72064B4FF440521A80FFF706FDC9
:10C20C00FEBD00BFCC090020600900200503002002
:10C21C00100D0020002383814FF416528380C380BD
:10C22C0003814FF00C030260438170470A8810B5FC
:10C23C004C88B1F804C0038AC98844EA020242EA75
:10C24C000C0223F470630A431B041B0C92B242EAE7
:10C25C000303038210BD00BF0023C380038043800F
:10C26C008380704721B183899BB243F4005304E06F
:10C27C00838923F400531B041B0C8381704700BF7C
:10C28C0001F01F034FF0010CC1F3421161450CFA90
:10C29C0003F301D10C3004E0022901D1103000E08D
:10C2AC0014301AB1026842EA030302E0026822EA7F
:10C2BC0003030360704700BF1AB1838A9BB2194312
:10C2CC0003E0838A9BB223EA01018182704700BF9D
:10C2DC00038A23F00F031B041B0C0382038A9BB2FB
:10C2EC0041EA030303827047838923F400631B0430
:10C2FC001B0C838183899BB241EA030383817047C2
:10C30C0021B183899BB243F0020304E0838923F0BB
:10C31C0002031B041B0C8381704700BF038A23F0AC
:10C32C0020031B041B0C0382038A9BB241EA030308
:10C33C000382704721B1038A9BB243F4804304E02B
:10C34C00038A23F480431B041B0C0382704700BF39
:10C35C00C905C90D818070478088C005C00D704724
:10C36C0083899BB243F0010383817047038BDBB25B
:10C37C000383038B9BB243EA01230383704700BF03
:10C38C00038B03F47F430383038B9BB241EA0303C8
:10C39C000383704721B1838A9BB243F0200304E0EE
:10C3AC00838A23F020031B041B0C8382704700BF7D
:10C3BC0021B1838A9BB243F0100304E0838A23F0FB
:10C3CC0010031B041B0C8382704700BF21B1838AAE
:10C3DC009BB243F0080304E0838A23F008031B0498
:10C3EC001B0C8382704700BF838A23F004031B0459
:10C3FC001B0C8382838A9BB241EA030383827047BE
:10C40C0021B1838A9BB243F0020304E0838A23F0B8
:10C41C0002031B041B0C8382704700BF0388194264
:10C42C000CBF002001207047C94389B201807047BE
:10C43C004FF0010CC1F3421201F01F0362450CFADC
:10C44C0003F301D1828903E0022A0CBF028A828A9B
:10C45C0092B21340028892B20BB9184607E0090A4F
:10C46C00012313FA01F111420CBF00200120704787
:10C47C00090A01238B40DB439BB20380704700BF4A
:10C48C00038ACA8823F440531B041B0C13430382F6
:10C49C0083898A8830B5044608890D4623F4B05345
:10C4AC00498940EA020223F00C030A431B041B0CCB
:10C4BC0092B242EA0303A381A38AAA8923F44073AC
:10C4CC001B041B0C134387B0A38201A801F0E8F8EE
:10C4DC000E4B2A689C420CBF049B039B19215943A9
:10C4EC0092006423B1FBF2F1B1FBF3F212011009DB
:10C4FC0003FB101109013231B1FBF3F303F00F030D
:10C50C0043EA020292B2228107B030BD00380140EA
:10C51C0008B5214B98422BD008D8A3F5006398425C
:10C52C0016D003F58063984234D119E01B4B984226
:10C53C0026D003F5684398422CD101214FF480405A
:10C54C0001F020F94FF48040002101F01BF921E0AB
:10C55C004FF40030012101F023F94FF4003016E0C4
:10C56C004FF48020012101F01BF94FF480200EE0E4
:10C57C004FF40020012101F013F94FF4002006E0E4
:10C58C004FF48010012101F00BF94FF480100021C1
:10C59C0001F006F908BD00BF004C004000500040FF
:10C5AC00038803F08F0303800388B1F806C04A8820
:10C5BC009BB243EA0C0313439BB203808B888385A5
:10C5CC000B880385064B984203D003F50063984211
:10C5DC0001D10B7A03864FF001038382704700BFB1
:10C5EC00002C0140038C2DE9F04123F001031B04C6
:10C5FC001B0C0384038C0A894C8823F002031C4E09
:10C60C0014431B048288B1F806C0058B1B0CA4B222
:10C61C00B04244EA030392B20C88ADB2A0F834C025
:10C62C0003D006F50066B04218D18E894F89B1F857
:10C63C000E804FF6F77C03EA0C0C4CEA070748EA2D
:10C64C0006064FF6FB73898847F6FF4C02EA0C0C82
:10C65C0007EA0303B2B20B4342EA0C024FF68F71A6
:10C66C0005EA01012143828001830384BDE8F08146
:10C67C00002C0140038C2DE9F04123F010031B0426
:10C68C001B0C0384028CB1F808C022F020021204A7
:10C69C008488120C4B8842EA0C1242EA0313A2B2B1
:10C6AC001B4C068BB1F806C0A0420D88B6B29BB2EB
:10C6BC00A0F838C003D004F50064A0421BD1B1F837
:10C6CC000A804FF67F748F8903EA040447F2FF3C1B
:10C6DC0002EA0C0C44EA0814CA894FF6BF73898825
:10C6EC0004EA03034CEA870C43EA01134CEA820286
:10C6FC003C469BB292B248F6FF7106EA010141EA50
:10C70C00052189B2828001830384BDE8F08100BFDA
:10C71C00002C0140038C2DE9F04123F480731B04A1
:10C72C001B0C0384028CB1F808C022F400721204B2
:10C73C008488120C4B8842EA0C2242EA0323A2B2F0
:10C74C001A4C868BB1F806C0A0420D88B6B29BB2CB
:10C75C00A0F83CC003D004F50064A0421BD1B1F892
:10C76C000A804FF2FF748F8903EA040444F6FF7CBD
:10C77C0002EA0C0C44EA0824CA894FF6FF33898874
:10C78C0004EA03034CEA071C43EA01234CEA0212B5
:10C79C003C469BB292B24FF68F7106EA01012943D7
:10C7AC00828081830384BDE8F08100BF002C0140AE
:10C7BC00038CF0B523F480531B041B0C0384B1F8D9
:10C7CC0006C0078C0C8882880D89868B4B88A0F854
:10C7DC0040C0DFF848C0BFB2604592B2B6B203D0D9
:10C7EC000CF5006C604505D192048989920C42EAE3
:10C7FC00811292B24DF6FF7C07EA0C0C48F6FF71E1
:10C80C0006EA01014CEA053C41EA04214CEA0333F7
:10C81C0089B29BB2828081830384F0BD002C0140DD
:10C82C00B1F802C00B888A884CEA0303B1F806C041
:10C83C0013430A8943EA0C03B1F80AC013438A89EB
:10C84C0043EA0C0313439BB2A0F84430704700BF7B
:10C85C0000234FF0FF320372438082800380C38039
:10C86C00704700BF0023C381038043808380C38053
:10C87C00038143818381704700234FF001020381C0
:10C88C00038043808280C380704700BF0023838174
:10C89C00038043808380C38003814381704700BF42
:10C8AC0021B103889BB243F0010304E0038823F019
:10C8BC0001039B059B0D0380704700BF39B1B0F895
:10C8CC0044306FEA43436FEA53439BB203E0B0F842
:10C8DC0044305B045B0CA0F8443070471AB1838978
:10C8EC009BB2194303E083899BB223EA0101818146
:10C8FC00704700BF818270470A43A0F848207047F8
:10C90C001AB183899BB2194303E083899BB223EA52
:10C91C0001018181704700BF038923F007031B04C9
:10C92C001B0C0381704700BFB0F808C05FFA8CFC89
:10C93C0041EA0C0C42EA0C0C4CEA032C1FFA8CFC5E
:10C94C00A0F808C0704700BF10B50446FFF7ECFF15
:10C95C0023899BB243F48043238110BD10B5044658
:10C96C00FFF7E2FF238923F077031B041B0C43F032
:10C97C007703238110BD00BF01858282704700BF01
:10C98C00038823F070039B059B0D41EA030303808E
:10C99C00704700BF038923F070031B041B0C41EA92
:10C9AC0003030381704700BF10B50446FFF7F2FF85
:10C9BC0023899BB243F00703238110BD30B5048952
:10C9CC00B0F818C0058C2CF4407CADB22CF0030CE4
:10C9DC0024F007044FEA0C4C25F0220542EA050529
:10C9EC0024044FEA1C4C45EA0315240C4CF4807CBF
:10C9FC0021434CF0010CADB20181A0F818C00584A4
:10CA0C0030BD00BF038B23F070031B041B0C41EAE9
:10CA1C0003030383704700BF038B23F4E0431B0421
:10CA2C001B0C43EA01239BB203837047838B23F0D7
:10CA3C0070031B041B0C41EA03038383704700BF84
:10CA4C00838B23F4E0431B041B0C43EA01239BB2AE
:10CA5C008383704721B103889BB243F0800304E0C9
:10CA6C00038823F080039B059B0D0380704700BF58
:10CA7C0021B183889BB243F0040304E0838823F044
:10CA8C0004031B041B0C8380704700BF21B18388F7
:10CA9C009BB243F0080304E0838823F008031B04D3
:10CAAC001B0C8380704700BF21B183889BB243F07D
:10CABC00010304E0838823F001031B041B0C838017
:10CACC00704700BF038B23F008031B041B0C41EAC7
:10CADC0003030383704700BF038B23F400631B0421
:10CAEC001B0C43EA01239BB203837047838B23F017
:10CAFC0008031B041B0C41EA03038383704700BF2C
:10CB0C00838B23F400631B041B0C43EA01239BB2AD
:10CB1C0083837047038B23F004031B041B0C41EA33
:10CB2C0003030383704700BF038B23F480631B0450
:10CB3C001B0C43EA01239BB203837047838B23F0C6
:10CB4C0004031B041B0C41EA03038383704700BFDF
:10CB5C00838B23F480631B041B0C43EA01239BB2DD
:10CB6C0083837047038B23F080031B041B0C41EA67
:10CB7C0003030383704700BF038B5B045B0C43EA26
:10CB8C0001239BB203837047838B23F080031B0428
:10CB9C001B0C41EA03038383704700BF838B5B0448
:10CBAC005B0C43EA01239BB283837047038C23F015
:10CBBC0002031B041B0C41EA03030384704700BFF0
:10CBCC00038C23F008031B041B0C41EA03030384AE
:10CBDC00704700BF038C23F020031B041B0C43EA9B
:10CBEC0001139BB203847047038C23F080031B0456
:10CBFC001B0C43EA01139BB203847047038C23F490
:10CC0C0000731B041B0C43EA01239BB20384704783
:10CC1C00038C23F400631B041B0C43EA01239BB21B
:10CC2C0003847047038C23F400531B041B0C43EA4E
:10CC3C0001339BB20384704701238B408A40018CE3
:10CC4C0089B221EA03030384018C0A4392B2028461
:10CC5C00704700BF04238B408A40018C89B221EAC3
:10CC6C0003030384018C0A4392B20284704700BF11
:10CC7C0001238B40B0F820C010B51FFA8CFC2CEAB5
:10CC8C000303038409B1082909D118304908445811
:10CC9C004FF68F7304EA0303435043580CE00439F6
:10CCAC001830C1F34E01445848F6FF7304EA0303ED
:10CCBC0043501202435892B243EA0202425010BD52
:10CCCC0021B103889BB243F0020304E0038823F0F4
:10CCDC0002039B059B0D0380704700BF21B10388A5
:10CCEC009BB243F0040304E0038823F004039B0588
:10CCFC009B0D0380704700BF21B183889BB243F02A
:10CD0C00800304E0838823F080031B041B0C8380C6
:10CD1C00704700BF038823F008039B059B0D03801D
:10CD2C0003889BB241EA030303807047838823F096
:10CD3C0070031B041B0C838083889BB241EA0303A2
:10CD4C0083807047038923F007031B041B0C0381AA
:10CD5C0003899BB241EA030303817047038923F0E3
:10CD6C0080031B041B0C038103899BB241EA030360
:10CD7C000381704781847047818570478186704735
:10CD8C000187704781877047A0F84010704700BF3B
:10CD9C00038B23F00C031B041B0C0383038B9BB230
:10CDAC0041EA030303837047038B23F440631B04A2
:10CDBC001B0C0383038B9BB243EA01239BB20383BB
:10CDCC00704700BF838B23F00C031B041B0C838365
:10CDDC00838B9BB241EA030383837047838B23F4D9
:10CDEC0040631B041B0C8383838B9BB243EA01239C
:10CDFC009BB28383704700BF0388DBB20380038838
:10CE0C009BB241EA03030380704700BF808E80B25F
:10CE1C00704700BF008F80B2704700BF808F80B218
:10CE2C00704700BFB0F8400080B27047808C80B271
:10CE3C00704700BF008D80B2704700BF038A194253
:10CE4C000CBF002001207047C94389B20182704792
:10CE5C00038A828911EA030092B203D011420CBFFB
:10CE6C0000200120704700BFC94389B2018270477E
:10CE7C00B0F820C010B52CF0010C4FEA0C4C4FEA66
:10CE8C001C4CA0F820C0048BB0F820C0A4B21FFA30
:10CE9C008CFC24F0F30442EA04042CF0020C44EA67
:10CEAC0003144CF0010C4CEA010CA4B20483A0F85E
:10CEBC0020C010BDB0F820C010B52CF0100C4FEAFB
:10CECC000C4C4FEA1C4CA0F820C0B0F818C0048CD5
:10CEDC002CF4407CA4B24FEA0C5C4FEA1C5C24F0AE
:10CEEC0020044CEA022C44F010044CEA033C44EAC3
:10CEFC0001141FFA8CFCA4B2A0F818C0048410BD55
:10CF0C0038B50D46602D1146044603D10122FFF7BA
:10CF1C00D1FF02E00122FFF7ABFF29462046FFF7C5
:10CF2C0039FD23899BB243F00703238138BD00BF31
:10CF3C00F8B50C46A2884988B4F800C0054600290B
:10CF4C000CBF02270027012A0CBF022601262389C9
:10CF5C00BCF1000F10D1FFF78BFF2846E188FFF7DB
:10CF6C0017FF2846394632462389FFF7A3FF284688
:10CF7C00E188FFF719FF0FE0FFF79CFF2846E188D7
:10CF8C00FFF712FF2846394632462389FFF770FF18
:10CF9C002846E188FFF7FCFEF8BD00BF38B50B88CA
:10CFAC000C4605464BB94988A2882389FFF760FFD8
:10CFBC002846E188FFF7ECFE53E0042B09D14988A1
:10CFCC00A2882389FFF776FF2846E188FFF7ECFE5D
:10CFDC0047E0082BB1F802C0B1F804E0098920D170
:10CFEC00028C22F480721204120C0284838B028C49
:10CFFC009BB292B223F0F30322F4007243EA0111C4
:10D00C0042EA0C2C89B21FFA8CFC41EA0E0E4CF44D
:10D01C00807CA0F81CE0A0F820C0E188FFF7D2FECD
:10D02C001FE0028C22F480521204120C0284838BB7
:10D03C00028C23F4407392B21B051B0D22F4005298
:10D04C0043EA0E2342EA0C3C43EA01331FFA8CFC00
:10D05C009BB24CF4805C8383A0F820C0E188FFF77E
:10D06C00BDFE38BD08B52D4B984237D00BD8A3F573
:10D07C000063984226D003F58063984228D0B0F123
:10D08C00804F4AD118E0264B984233D004D8A3F5F0
:10D09C008063984241D127E0224B984204D003F59B
:10D0AC000063984239D12EE04FF40060012100F06A
:10D0BC0069FB4FF400602DE00120014600F070FB8D
:10D0CC0001201CE00220012100F06AFB022016E086
:10D0DC000420012100F064FB042010E00820012151
:10D0EC0000F05EFB08200AE01020012100F058FB44
:10D0FC00102004E02020012100F052FB2020002110
:10D10C0000F04EFB09E04FF40050012100F03AFB17
:10D11C004FF40050002100F035FB08BD000C00401E
:10D12C0000140040002C0140042804D1054B1A685F
:10D13C0042F0040203E0034B1A6822F004021A6066
:10D14C00704700BF10E000E0014B5860704700BF13
:10D15C0010E000E0012804D1084B1A6842F00102EB
:10D16C0006E010F1020F05D1044B1A6822F00102FF
:10D17C001A6002E0014B00229A60704710E000E058
:10D18C0020B1054B1A6842F0020203E0024B1A6808
:10D19C0022F002021A60704710E000E0014B986820
:10D1AC00704700BF10E000E0C308022B0BBF044B1C
:10D1BC00034B1B68DB6833FA00F000F0010070478A
:10D1CC0010E000E00B884A88B1F804C01A43CB8801
:10D1DC0042EA0C02B1F808C01A434B8930B542EA56
:10D1EC000C028D89B0F800C0CC891A432A43224323
:10D1FC000CF4415313439BB20380838B23F40063E1
:10D20C001B041B0C83830B8A038230BD00234FF05D
:10D21C000702C3810282038043808380C380038121
:10D22C0043818381704700BF002343810380438087
:10D23C008380C3804FF002030381704721B10388C0
:10D24C009BB243F0400304E0038823F040031B042B
:10D25C001B0C0380704700BF21B1838B9BB243F43E
:10D26C00806304E0838B23F480631B041B0C838397
:10D27C00704700BF0909012313FA01F189B21AB1F1
:10D28C0083889BB2194303E083889BB223EA010194
:10D29C00818070471AB183889BB2194303E083885D
:10D2AC009BB223EA01018180704700BF81817047E6
:10D2BC00808980B2704700BF4FF6FF63994205D05A
:10D2CC0003889BB243F48073038002E00388194007
:10D2DC000180704721B183889BB243F0040304E0C2
:10D2EC00838823F004031B041B0C8380704700BF4E
:10D2FC00038823F400631B041B0C038003889BB27C
:10D30C0041EA03030380704703889BB243F48053C4
:10D31C000380704721B103889BB243F4005304E0AF
:10D32C00038823F400531B041B0C0380704700BFBD
:10D33C00012914BF008B808A80B27047008A80B2AA
:10D34C00704700BFB1F5804F04D103889BB243F402
:10D35C00804304E0038823F480431B041B0C0380EC
:10D36C00704700BF038919420CBF00200120704791
:10D37C00202906D1038903889BB243F04003038024
:10D38C0008E0402901D0082901D1038902E0C943F2
:10D39C0089B20181704700BF012301F00F0213FA1B
:10D3AC0002F2B0F804C000891FFA8CFC80B2104065
:10D3BC0006D009098B401CEA030F0CBF002001208A
:10D3CC00704700BF552906D1038903889BB243F0EF
:10D3DC00400303800DE0562901D0532901D1038964
:10D3EC0007E001F00F01012313FA01F1C94389B2DF
:10D3FC0001817047838BF0B523F47A6323F01F030C
:10D40C001B041B0C83834FF0020303840B89868B54
:10D41C00022B87B004460D46B6B201D1002225E09E
:10D42C0001A88F8800F03CF9EB88002F0CBF012776
:10D43C000227B3F5007F2989019A06D1A3F5FB7366
:10D44C0053430902B3FBF1F305E00A2349015A43A4
:10D45C004F43B2FBF7F305330A229BB2B3FBF2F353
:10D46C0003F001021202C3F34F0392B2991E89B268
:10D47C00FE2928BF002228BF0223E98842EA0303C1
:10D48C000B439BB223842B886A8846EA0303A98842
:10D49C0043F4006313436A890B4313439BB2A38386
:10D4AC0007B0F0BD08B5154B98421BD003F574437B
:10D4BC00984204D0A3F5784398421DD10AE001218B
:10D4CC004FF4805000F05EF94FF48050002100F0D2
:10D4DC0059F911E04FF48040012100F061F94FF44B
:10D4EC00804006E04FF40040012100F059F94FF460
:10D4FC000040002100F054F908BD00BF003C004082
:10D50C000D4B0E4A196841F001011960596801EA86
:10D51C0002025A601A6822F0847222F480321A6075
:10D52C001A6822F480221A605A6822F4FE025A60A9
:10D53C0000229A60704700BF001002400000FFF804
:10D54C000C4BB0F5803F1A6822F480321A601A68CE
:10D55C0022F480221A6003D0B0F5802F08D103E0AA
:10D56C001A6842F4803202E01A6842F4A0221A606F
:10D57C00704700BF00100240034B1A6822F0F802FB
:10D58C0042EAC0021A60704700100240014B18605A
:10D59C00704700BF00004242044B5A6822F47C12D0
:10D5AC0040EA02020A435A60704700BF0010024072
:10D5BC00014B1860704700BF60004242034B5A6831
:10D5CC0022F0030240EA02025A6070470010024047
:10D5DC00024B586800F00C00704700BF001002406E
:10D5EC00034B5A6822F0F00240EA02025A6070477C
:10D5FC0000100240034B5A6822F4E06240EA020237
:10D60C005A60704700100240034B5A6822F4605273
:10D61C0042EAC0025A6070470010024019B1054B33
:10D62C001A78104303E0034B1A7822EA00001870B2
:10D63C00704700BF09100240014B1860704700BFD3
:10D64C00D8004242034B5A6822F4404240EA02029C
:10D65C005A60704700100240064B002201281A70D5
:10D66C001A7002D0042804D101E0187001E00522E0
:10D67C001A70704720100240014B1860704700BFB1
:10D68C0080044242024B1A6A40EA02021A62704754
:10D69C0000100240014B1860704700BF3C0442422E
:10D6AC001F4B10B55A6802F00C02042A13D0082A3A
:10D6BC0011D15A685968C2F38342023211F4803F87
:10D6CC0003D05B6813F4003F01D0164B00E0164BFF
:10D6DC005A43026001E0144B0360114A134B51682A
:10D6EC000468C1F30311595C34FA01F141605468C8
:10D6FC00C4F3022C13F80C4031FA04F4846054681F
:10D70C00C4F3C22C13F80CC021FA0CF1C16052689E
:10D71C00C2F381329B181B7CB1FBF3F1016110BD8C
:10D72C000010024000093D0000127A00F8F90008D0
:10D73C0019B1054B5A69104303E0034B5A6922EAAD
:10D74C0000005861704700BF0010024019B1054B32
:10D75C009A69104303E0034B9A6922EA000098612E
:10D76C00704700BF0010024019B1054BDA69104335
:10D77C0003E0034BDA6922EA0000D861704700BF6E
:10D78C000010024019B1054BDA68104303E0034B5B
:10D79C00DA6822EA0000D860704700BF001002402F
:10D7AC0019B1054B1A69104303E0034B1A6922EABD
:10D7BC0000001861704700BF00100240014B186058
:10D7CC00704700BF40044242014B1860704700BFD5
:10D7DC004C004242014B1870704700BF07100240CA
:10D7EC004309012B02D1084B1B6805E0022B0BBF30
:10D7FC00054B054B1B6A5B6A00F01F0033FA00F007
:10D80C0000F00100704700BF0010024008B5312045
:10D81C00FFF7E6FF094B18705A6801325A601A7804
:10D82C0022B95A6840F2FF139A42F0D13120FFF727
:10D83C00D7FF003818BF012008BD00BF0803002027
:10D84C00024B5A6A42F080725A62704700100240D2
:10D85C00034B9B6818420CBF00200120704700BF8F
:10D86C0000100240014B1870704700BF0A100240B4
:10D87C000B4B4FF0FF316FF07042C3F88010C3F8C0
:10D88C008420C3F88011C3F88421002303F1C00164
:10D89C00034A013300200F2B42F82100F6D17047C8
:10D8AC0000E100E0094B4FF020605860084800226E
:10D8BC004FF0FF319A60D8601A615A619A61DA614F
:10D8CC001A625A629962D9621963704700ED00E0DE
:10D8DC000000FA0540F0BE60024B40F42020D860F6
:10D8EC00704700BF00ED00E030B5C27803787AB322
:10D8FC001C4A4178D2684FF00F0CD243C2F302227B
:10D90C002CFA02FCC2F104029140807803F003026D
:10D91C000CEA000C4CEA010CD2004FEA0C1CFF2064
:10D92C0090400CFA02FC012403F01F029440990869
:10D93C000D4AC03152F821500CEA000C25EA0000C7
:10D94C004CEA00005B0942F8210042F8234008E051
:10D95C0003F01F02012191405B09034A203342F876
:10D96C00231030BD00ED00E000E100E00023C370A7
:10D97C000370437083707047024B5868C0F30930D2
:10D98C00704700BF00ED00E0012200F01F0312FA07
:10D99C0003F34009044A403052F8200018409842E2
:10D9AC0014BF00200120704700E100E0014B18601B
:10D9BC00704700BF00EF00E000F01F0301229A4007
:10D9CC004009024B603043F82020704700E100E032
:10D9DC00024B58688005800D704700BF00ED00E0D9
:10D9EC00012200F01F0312FA03F34009044A8030AD
:10D9FC0052F820001840984214BF002001207047B4
:10DA0C0000E100E0014B1868704700BF00ED00E03A
:10DA1C0021F0604121F07F01014B01439960704777
:10DA2C0000ED00E0014A024BDA6070470400FA0591
:10DA3C0000ED00E0014A024BDA6070470100FA0584
:10DA4C0000ED00E019B1054B1A69104303E0034BDC
:10DA5C001A6922EA00001861704700BF00ED00E06F
:10DA6C0000F01F00012313FA00F019B1044B5A6A9D
:10DA7C00104303E0024B5A6A22EA000058627047D6
:10DA8C0000ED00E0144B70B5DC684FF0FF0CE44384
:10DA9C00C4F302242CFA04F5C4F1040411FA04F4BE
:10DAAC00C0F30126F6000CFA06FC02EA050545EA6D
:10DABC000404240114FA06F6C0F38110063053F85E
:10DACC00202022EA0C0243F8202053F82020164391
:10DADC0043F8206070BD00BF00ED00E0C0F3832070
:10DAEC0001238340044A506A03EA0000984214BFA1
:10DAFC0000200120704700BF00ED00E000F01F0087
:10DB0C0001228240024B59680A435A60704700BF99
:10DB1C0000ED00E000F01F020123013A13FA02F2BB
:10DB2C00024B59680A435A60704700BF00ED00E091
:10DB3C00C0F3833001238340044A506A03EA000097
:10DB4C00984214BF00200120704700BF00ED00E098
:10DB5C00C0F3814313B90A4BD86A10E0012B0CD1E6
:10DB6C00074AC0F30153906ADA00D040022B14BF6D
:10DB7C0000F00F0000F0FF0001E0014B186B704744
:10DB8C0000ED00E010F4800F0BBF024B014B586B03
:10DB9C00986B704700ED00E008B5F6F7E1FA08BDA8
:10DBAC0008B50001F6F7D9FA08BD00BF08B5F6F7BD
:10DBBC00D2FA08BD08B5F6F7CCFA08BD08B5F6F7E9
:10DBCC00C6FA08BD08B5F6F7C0FA08BDCB78F0B5B3
:10DBDC0013F0100F18BF8A78098803F00F0C18BFC8
:10DBEC004CEA020C11F0FF0F1AD004680022012637
:10DBFC00964006EA0105B5420ED196000F27B740B4
:10DC0C000CFA06F624EA07043443282B01D14561AB
:10DC1C0002E0482B08BF05610132082AE7D10460F5
:10DC2C00FF291CD94468002202F108050126AE40E8
:10DC3C0006EA0105B5420ED196000F27B7400CFA43
:10DC4C0006F624EA07043443282B01D1456102E08F
:10DC5C00482B08BF05610132082AE5D14460F0BDAC
:10DC6C000423C370022383704FF0FF33038070478B
:10DC7C00836819420CBF002001207047806880B275
:10DC8C00704700BFC36819420CBF002001207047C9
:10DC9C00C06880B2704700BF016170474161704736
:10DCAC000AB1016100E04161704700BFC16070477B
:10DCBC0041F4803383618161836183698369704737
:10DCCC00064A10B514684FF6807341EA001104EA55
:10DCDC00030341EA0303136010BD00BF00000140C1
:10DCEC00014B1860704700BF1C0020420304154A0A
:10DCFC0000F4401C1B0CBCF5401F30B5546806D119
:10DD0C00556824F0706425F07065556011E010F4CE
:10DD1C00801F06D0C0F303424FF0030C0CFA02F242
:10DD2C0003E0420D120113FA02F224EA020444F059
:10DD3C00706419B1400D000183401C43014B5C60C1
:10DD4C0030BD00BF0000014001F003039B000F2217
:10DD5C009A4010FA03F310B58908074C023154F8B5
:10DD6C00210020EA020244F8212054F82120134318
:10DD7C0044F8213010BD00BF0000014001200146D5
:10DD8C0008B5FFF7FFFC01200021FFF7FBFC08BDE5
:10DD9C0008B5264B98422BD00CD8A3F500639842BB
:10DDAC001AD003F5806398421CD0A3F50063984207
:10DDBC003AD10BE01E4B984226D003F58063984273
:10DDCC0028D0A3F5006398422ED117E0042001213E
:10DDDC00FFF7D8FC042024E008200121FFF7D2FC37
:10DDEC0008201EE010200121FFF7CCFC102018E0C9
:10DDFC0020200121FFF7C6FC202012E04020012149
:10DE0C00FFF7C0FC40200CE080200121FFF7BAFC9A
:10DE1C00802006E04FF480700121FFF7B3FC4FF433
:10DE2C0080700021FFF7AEFC08BD00BF001401405C
:10DE3C00001C0140044B1A6802F038021A601A6880
:10DE4C0040EA02021A60704700200240044B1A6834
:10DE5C0022F008021A601A6840EA02021A6070473F
:10DE6C0000200240044B1A6822F010021A601A6853
:10DE7C0040EA02021A60704700200240044B002264
:10DE8C001A605A609A60DA60024A5A61704700BFA1
:10DE9C0000040140FFFF0700837930B50168027967
:10DEAC004BB3184BCC431D6890F805C004EA05052C
:10DEBC001D605D682C405C60D45844EA0101D1506F
:10DECC0002689868D14301EA00009860D868014064
:10DEDC00BCF1100FD96007D1996811439960D968CA
:10DEEC0041EA0202DA600BE05CF8031041EA02023C
:10DEFC004CF8032004E0034BD05820EA0101D15028
:10DF0C0030BD00BF0004014000230C22837142711C
:10DF1C0003600371704700BF024B1A6940EA0202AA
:10DF2C001A61704700040140034B5B6918420CBF37
:10DF3C0000200120704700BF00040140014B5861D4
:10DF4C00704700BF00040140054B1A685B69034031
:10DF5C0001D1184603E010420CBF0020012070478D
:10DF6C0000040140014B5861704700BF00040140A0
:10DF7C000268002322F001020260036043608360A8
:10DF8C00C3602D4B984233D011D83C3B984229D0DA
:10DF9C0006D8283B984221D0143398424BD11FE02D
:10DFAC00264B984220D01433984244D11EE0244B87
:10DFBC0098422CD008D8A3F5677398421DD003F56E
:10DFCC006273984237D11DE01E4B984229D014330E
:10DFDC0098422BD0283B98422DD11DE01A4B12E0D1
:10DFEC00194B15E0184B18E0174B1BE0164B1EE0B5
:10DFFC00154B5A6842F470021CE0134B5A6842F0FD
:10E00C00706217E0114B5A6842F00F0212E00F4B8E
:10E01C005A6842F0F0020DE00C4B5A6842F4706200
:10E02C0008E00A4B5A6842F4704203E0074B5A6806
:10E03C0042F470225A6070476C0002404400024067
:10E04C001C04024044040240000002400004024050
:10E05C008A6870B50C6A0B6944EA02024C691A436F
:10E06C008B692243CC6905684E6A42EA0303234359
:10E07C008C6A334325F4FE4C23432CF0F00C43EA1A
:10E08C000C030360CB6843600B6883604B68C36010
:10E09C0070BD00BF00238362036043608360C36074
:10E0AC00036143618361C36103624362704700BFD4
:10E0BC0019B1036843F0010302E0036823F0010384
:10E0CC000360704712B10368194302E0036823EA46
:10E0DC0001010160704700BF406880B2704700BF0B
:10E0EC0010F0805F14BF044B044B1B6803420CBF41
:10E0FC0000200120704700BF0004024000000240D5
:10E10C0010F0805F14BF024B024B5860704700BF89
:10E11C00000402400000024010F0805F14BF044B6A
:10E12C00044B1B6803420CBF00200120704700BF4A
:10E13C00000402400000024010F0805F14BF024B4C
:10E14C00024B5860704700BF0004024000000240C0
:10E15C00374B01221A605A6812F0010201D11046A5
:10E16C0064E00278012A0BBF1A681A6842F0800238
:10E17C0022F080021A604378012B04D12C4B1A68D0
:10E18C0042F0400203E02A4B1A6822F040021A6067
:10E19C008378012B04D1264B1A6842F0200203E04D
:10E1AC00234B1A6822F020021A60C378012B04D189
:10E1BC001F4B1A6842F0100203E01D4B1A6822F044
:10E1CC0010021A600379012B04D1194B1A6842F022
:10E1DC00080203E0164B1A6822F008021A60437911
:10E1EC00012B04D1124B1A6842F0040203E0104BCD
:10E1FC001A6822F004021A608279C37990F808C078
:10E20C00920742EA03624189437A42EA0C4242EAAB
:10E21C0003520139064B0A43DA611A6822F00102F3
:10E22C001A60586880F0010000F00100704700BFD0
:10E23C000064004090F800C0012202FA0CF23B4B43
:10E24C002DE9F045D3F8004292B244F00104C3F832
:10E25C000042D3F81C42D14301EA0404C3F81C4227
:10E26C008478A4B90CF1480CD3F80C72B0F80AA05D
:10E27C00C688B0F8088085884FEACC0404F1804445
:10E28C0046EA0A4645EA084501EA070715E0012C6B
:10E29C001AD10CF1480CD3F80C72B0F804A0C68853
:10E2AC00B0F8088045894FEACC0404F1804446EA72
:10E2BC000A4645EA084542EA070704F5C844C3F88C
:10E2CC000C7243F83C60656043782BB9174BD3F85C
:10E2DC00044201EA040404E0144BD3F8044242EA79
:10E2EC000404C3F80442838923B9104BD3F81442B5
:10E2FC00214006E0012B06D10C4BD3F8141242EA54
:10E30C000101C3F81412837B012B05D1074BD3F801
:10E31C001C120A43C3F81C22044BD3F8002222F02F
:10E32C000102C3F80022BDE8F08500BF0064004084
:10E33C0003220272013A002342724FF00102C371B0
:10E34C004281037043708370C37003714371837196
:10E35C00704700BF19B1054B5A69104303E0034BDA
:10E36C005A6922EA00005861704700BF00640040FF
:10E37C00364B70B59968024611F0806F01D00020C1
:10E38C000CE0996811F0006F01D0012006E09B6849
:10E39C0013F0805F01D1042056E002202B4B00F1DA
:10E3AC0018010901CC5804F00104CC50157A92F8EC
:10E3BC0009C035B9146864051460CD584CEA050CD5
:10E3CC0007E0546845EA0C0CE4005460CE584CEA63
:10E3DC00060C4CEA0404CC50947A00F1180C4FEA69
:10E3EC000C1C04F00F040CF18043947203F5C84329
:10E3FC005D68010125F00F055D605D6801F18041EC
:10E40C002C435C60537B947BD57A1B0443EA0463F6
:10E41C00147B2B4343EA042301F5C841C1F888312E
:10E42C00557C937CD47B2D0445EA0365137C45EA2B
:10E43C00040242EA0322054BC1F88C215CF803204C
:10E44C0042F001024CF8032070BD00BF0064004094
:10E45C00012810D002D302282CD11AE0164A916858
:10E46C009368926801F0010103F0020343EA81030F
:10E47C00C2F380621AE0104A9368916803F48073C7
:10E48C00926801F400719B0943EA1123C2F3C06244
:10E49C000CE0094A9368916803F48033926801F4A4
:10E4AC0000319B0B43EA1143C2F300721343034A3E
:10E4BC00D05C70470023FAE7006400400CFA0008B7
:10E4CC00012808D002D302280FD109E0074B9A6823
:10E4DC0042F0800208E0054B9A6842F4004203E0E7
:10E4EC00024B9A6842F400029A6070470064004044
:10E4FC0018B9044B2022DA6002E0024B20221A6188
:10E50C00704700BF0064004010B9064BD86805E0A6
:10E51C00012801D0002003E0024B186900F0030031
:10E52C00704700BF00640040254B00F11B02120134
:10E53C0010B5D45804F004040C721CB9D3585B0DFC
:10E54C000B6002E0D358DB084B6000F11B021C4B44
:10E55C001201D35802F1804203F002034B7202F510
:10E56C00C8425468030104F00F0C81F80AC05268C9
:10E57C0003F18043120ACA7403F5C843D3F8B821D7
:10E58C00CA72D3F8B821120A0A73D3F8B821120C44
:10E59C004A73D3F8B821120E8A73D3F8BC21CA730C
:10E5AC00D3F8BC21120A0A74D3F8BC21120C4A7499
:10E5BC00D3F8BC311B0E8B74FFF79AFF10BD00BF54
:10E5CC0000640040044B1A6842F002021A6018689A
:10E5DC00C0F34000704700BF00640040054B1A6850
:10E5EC0022F002021A60186880F00200C0F34000AA
:10E5FC00704700BF00640040034B9B6918420CBF7E
:10E60C0000200120704700BF00640040024B9A6953
:10E61C0022EA00029A61704700640040202831D041
:10E62C000CD8062820D004D8042825D0052844D19D
:10E63C0018E007281DD008283FD11FE0B0F5007F57
:10E64C002BD005D840281FD0B0F5807F35D11FE0E6
:10E65C00B0F5803F2CD0B0F5003F2BD0B0F5806FDB
:10E66C002BD11FE0012201E04FF48072134B9A6012
:10E67C0023E04FF48032F9E7082200E010220F4B20
:10E68C00DA601AE0082200E010220C4B1A6114E048
:10E69C000A4B9A6922F0010208E0084B9A6922F0B1
:10E6AC00020203E0054B9A6922F004029A6104E02D
:10E6BC00082200E01022014B5A60704700640040B1
:10E6CC0001420CBF00200120704700BF202808B574
:10E6DC0032D00CD8062821D004D8042826D00528FE
:10E6EC0018D119E007281ED0082813D120E0B0F566
:10E6FC00007F29D005D8402820D0B0F5807F09D1E3
:10E70C0020E0B0F5803F27D0B0F5003F22D0B0F527
:10E71C00806F1BD0002024E0012101E04FF48071B8
:10E72C00104B98681BE04FF48031F9E7082100E0AA
:10E73C0010210C4BD86812E0082100E01021094B85
:10E74C0018690CE0012102E0022100E00421054BD4
:10E75C00986904E0102100E00821024B5868FFF78B
:10E76C00AFFF08BD00640040012108B54FF00070F8
:10E77C00FFF716F84FF000700021FFF711F808BDF5
:10E78C00436830B523F470230C680A7923F4807342
:10E79C00234343EA0223436082688D68CC680A4BAA
:10E7AC0045EA040C02EA03034A794CEA030343EA00
:10E7BC00420383600B7CC26A013B22F47002DBB221
:10E7CC0042EA0353C36230BDFDF7F1FF002301227F
:10E7DC000274C3600360037143718360704700BFB0
:10E7EC0019B1836843F0010302E0836823F001034D
:10E7FC008360704719B1836843F4807302E08368C7
:10E80C0023F4807383607047C9B212B14368194313
:10E81C0002E0436823EA010141607047836843F0DA
:10E82C0008038360704700BF8068C0F3C000704766
:10E83C00836843F004038360704700BF8068C0F3B3
:10E84C008000704719B1836843F4A00302E0836829
:10E85C0023F4A003836070478068C0F38050704736
:10E86C004368013923F4604343EA41334360704702
:10E87C0019B1436843F4006302E0436823F4006376
:10E88C0043607047092930B511D94FF0030C0CFBCC
:10E89C0001FC0725ACF11E0C05FA0CF503FA0CFC77
:10E8AC00C46824EA050343EA0C03C3600EE04FF08E
:10E8BC00030C0CFB01FC072505FA0CF503FA0CFC08
:10E8CC00046924EA050343EA0C030361062A0DD804
:10E8DC000523013A5A434FF01F0C0CFA02FC9140ED
:10E8EC00436B23EA0C020A4342631CE00C2A0DD84A
:10E8FC0005235A434FF01F0C233A0CFA02FC9140AB
:10E90C00036B23EA0C020A4302630CE005235A430F
:10E91C004FF01F0C413A0CFA02FC9140C36A23EAF7
:10E92C000C020A43C26230BD19B1836843F48013F0
:10E93C0002E0836823F4801383607047C06C80B25C
:10E94C00704700BF014B1868704700BF4C24014052
:10E95C0019B1436843F4806302E0436823F4806395
:10E96C004360704719B1436843F4805302E0436835
:10E97C0023F4805343607047836823F4E04341EAF7
:10E98C0003038360704700BF19B1836843F40043ED
:10E99C0002E0836823F400438360704719B18368F5
:10E9AC0043F4021302E0836823F40213836070477C
:10E9BC008068C0F340507047092930B511D94FF029
:10E9CC00030C0CFB01FC0725ACF11E0C05FA0CF535
:10E9DC0003FA0CFCC46824EA050343EA0C03C36085
:10E9EC000EE04FF0030C0CFB01FC072505FA0CF5AF
:10E9FC0003FA0CFC046924EA050343EA0C030361E3
:10EA0C00836BC3F3015CCCEB020202324FF0050CBA
:10EA1C00D2B20CFB02F20CF11A0C0CFA02FC914073
:10EA2C0023EA0C030B43836330BD00BF836B0139B6
:10EA3C0023F4401343EA0153836370470A50704731
:10EA4C002830405880B27047436823F4400323F4C5
:10EA5C00007341EA03034360704700BF4162826266
:10EA6C00704700BF436823F01F0341EA0303436070
:10EA7C00704700BF20B1054B9A6842F4000203E0D6
:10EA8C00024B9A6822F400029A60704700240140FD
:10EA9C00036819420CBF002001207047C943016074
:10EAAC00704700BF4368006810EA112004D0C9B257
:10EABC0019420CBF00200120704700BF6FEA1121E2
:10EACC000160704708B5134B98420FD003F5A05363
:10EADC00984213D0A3F5C053984219D14FF400704B
:10EAEC000121FEF74FFE4FF400700EE04FF48060F2
:10EAFC000121FEF747FE4FF4806006E04FF4004022
:10EB0C000121FEF73FFE4FF400400021FEF73AFED4
:10EB1C0008BD00BF00280140032A2DE9F0070BD8DF
:10EB2C003AB1002311F803C000F803C0013393423B
:10EB3C00F8D1BDE8F007704782180C46034603E095
:10EB4C0014F8011C03F8011C03F003061946A44633
:10EB5C0001330134002EF3D11CF00304634608BFCB
:10EB6C00C1EB020C68D06542C4F1040A0CEB05073A
:10EB7C0033464FEACA0A5CF805604FEAC408551AD6
:10EB8C0008E057F8044F264604FA0AF449EA04044C
:10EB9C00CC5004335C18032D26FA08F9A5F10405B2
:10EBAC000CEB0306EDDC002302E0F15CE1540133D5
:10EBBC0019199142F9D3BCE753F8404C41F8404C39
:10EBCC0053F83C4C41F83C4C53F8384C41F8384C19
:10EBDC0053F8344C41F8344C53F8304C41F8304C29
:10EBEC0053F82C4C41F82C4C53F8284C41F8284C39
:10EBFC0053F8244C41F8244C53F8204C41F8204C49
:10EC0C0053F81C4C41F81C4C53F8184C41F8184C58
:10EC1C0053F8144C41F8144C53F8104C41F8104C68
:10EC2C0053F80C4C41F80C4C53F8084C41F8084C78
:10EC3C0053F8044C41F8044C1C460D46403340310B
:10EC4C00BCF13F0FACF1400CB6DC21462B46541BFB
:10EC5C000FE051F8105C43F8105C51F80C5C43F871
:10EC6C000C5C51F8085C43F8085C51F8045C43F800
:10EC7C00045C0F2C0D469C4601F1100103F11003AE
:10EC8C00A4F11004E5DCCCEB0201002303E0EC580A
:10EC9C004CF8034004335E19032903EB0C04A1F177
:10ECAC000401F4DC7FE700BF80F0004002E000BF0D
:10ECBC0081F0004142001FBF5FEA410392EA030F5B
:10ECCC007FEA226C7FEA236C6AD04FEA1262D2EBA5
:10ECDC001363C1BFD218414048404140B8BF5B42AA
:10ECEC00192B88BF704710F0004F40F4000020F043
:10ECFC007F4018BF404211F0004F41F4000121F059
:10ED0C007F4118BF494292EA030F3FD0A2F10102A2
:10ED1C0041FA03FC10EB0C00C3F1200301FA03F1E0
:10ED2C0000F0004302D5494260EB4000B0F5000F03
:10ED3C0013D3B0F1807F06D340084FEA310102F1C2
:10ED4C000102FE2A51D2B1F1004F40EBC25008BF74
:10ED5C0020F0010040EA03007047490040EB00003E
:10ED6C0010F4000FA2F10102EDD1B0FA80FCACF16D
:10ED7C00080CB2EB0C0200FA0CF0AABF00EBC2506C
:10ED8C0052421843BCBFD0401843704792F0000F5A
:10ED9C0081F4000106BF80F400000132013BB5E7AD
:10EDAC004FEA41037FEA226C18BF7FEA236C21D023
:10EDBC0092EA030F04D092F0000F08BF0846704788
:10EDCC0090EA010F1CBF0020704712F07F4F04D156
:10EDDC00400028BF40F00040704712F100723CBF69
:10EDEC0000F50000704700F0004343F0FE4040F493
:10EDFC00000070477FEA226216BF08467FEA236351
:10EE0C000146420206BF5FEA412390EA010F40F43B
:10EE1C00800070474FF0000304E000BF10F0004387
:10EE2C0048BF40425FEA000C08BF704743F096436E
:10EE3C0001464FF000001CE050EA010208BF704789
:10EE4C004FF000030AE000BF50EA010208BF704710
:10EE5C0011F0004302D5404261EB41015FEA010C25
:10EE6C0002BF84460146002043F0B64308BFA3F11D
:10EE7C008053A3F50003BCFA8CF2083AA3EBC253FF
:10EE8C0010DB01FA02FC634400FA02FCC2F120021E
:10EE9C00BCF1004F20FA02F243EB020008BF20F055
:10EEAC000100704702F1200201FA02FCC2F12002BB
:10EEBC0050EA4C0021FA02F243EB020008BF20EAB0
:10EECC00DC7070474FF0FF0C1CEAD0521EBF1CEADE
:10EEDC00D15392EA0C0F93EA0C0F6FD01A4480EACC
:10EEEC00010C400218BF5FEA41211ED04FF00063B5
:10EEFC0043EA501043EA5111A0FB01310CF00040E1
:10EF0C00B1F5000F3EBF490041EAD3715B0040EA06
:10EF1C00010062F17F02FD2A1DD8B3F1004F40EBD6
:10EF2C00C25008BF20F00100704790F0000F0CF0A9
:10EF3C00004C08BF49024CEA502040EA51207F3A6D
:10EF4C00C2BFD2F1FF0340EAC250704740F4000048
:10EF5C004FF00003013A5DDC12F1190FDCBF00F039
:10EF6C0000407047C2F10002410021FA02F1C2F1E7
:10EF7C00200200FA02FC5FEA310040F1000053EA83
:10EF8C004C0308BF20EADC70704792F0000F00F0D1
:10EF9C00004C02BF400010F4000F013AF9D040EAD7
:10EFAC000C0093F0000F01F0004C02BF490011F46B
:10EFBC00000F013BF9D041EA0C018FE70CEAD15369
:10EFCC0092EA0C0F18BF93EA0C0F0AD030F0004CE9
:10EFDC0018BF31F0004CD8D180EA010000F000409D
:10EFEC00704790F0000F17BF90F0004F084691F05B
:10EFFC00000F91F0004F14D092EA0C0F01D1420295
:10F00C000FD193EA0C0F03D14B0218BF084608D15D
:10F01C0080EA010000F0004040F0FE4040F40000A7
:10F02C00704740F0FE4040F4400070474FF0FF0C3A
:10F03C001CEAD0521EBF1CEAD15392EA0C0F93EA81
:10F04C000C0F69D0A2EB030280EA010C49024FEAD3
:10F05C00402037D04FF0805343EA111143EA10138C
:10F06C000CF000408B4238BF5B0042F17D024FF444
:10F07C00000C8B4224BF5B1A40EA0C00B3EB510F1F
:10F08C0024BFA3EB510340EA5C00B3EB910F24BF08
:10F09C00A3EB910340EA9C00B3EBD10F24BFA3EB8D
:10F0AC00D10340EADC001B0118BF5FEA1C1CE0D155
:10F0BC00FD2A3FF650AF8B4240EBC25008BF20F008
:10F0CC00010070470CF0004C4CEA50207F32C2BF5C
:10F0DC00D2F1FF0340EAC250704740F400004FF0F9
:10F0EC000003013A37E792F0000F00F0004C02BF2A
:10F0FC00400010F4000F013AF9D040EA0C0093F0F4
:10F10C00000F01F0004C02BF490011F4000F013B4D
:10F11C00F9D041EA0C0195E70CEAD15392EA0C0FB5
:10F12C0008D142027FF47DAF93EA0C0F7FF470AFED
:10F13C00084676E793EA0C0F04D14B023FF44CAF30
:10F14C0008466EE730F0004C18BF31F0004CCAD1C5
:10F15C0030F000427FF45CAF31F000437FF43CAF01
:10F16C005FE700BF4FF0FF3C06E000BF4FF0010C23
:10F17C0002E000BF4FF0010C4DF804CD4FEA400205
:10F18C004FEA41037FEA226C18BF7FEA236C11D04F
:10F19C0001B052EA530C18BF90EA010F58BFB2EB02
:10F1AC00030088BFC81738BF6FEAE17018BF40F082
:10F1BC00010070477FEA226C02D15FEA402C05D136
:10F1CC007FEA236CE4D15FEA412CE1D05DF8040BBB
:10F1DC00704700BF844608466146FFE70FB5FFF74E
:10F1EC00C9FF002848BF10F1000F0FBD4DF808ED06
:10F1FC00FFF7F4FF0CBF012000205DF808FB00BFF7
:10F20C004DF808EDFFF7EAFF34BF012000205DF850
:10F21C0008FB00BF4DF808EDFFF7E0FF94BF01209D
:10F22C0000205DF808FB00BF4DF808EDFFF7D2FF9A
:10F23C0094BF012000205DF808FB00BF4DF808EDDD
:10F24C00FFF7C8FF34BF012000205DF808FB00BFAA
:10F25C004FEA4002B2F1FE4F0FD34FF09E03B3EBD7
:10F26C0012620DD94FEA002343F0004310F0004F17
:10F27C0023FA02F018BF404270474FF0000070476D
:10F28C0012F1610F01D1420205D110F0004008BF0C
:10F29C006FF0004070474FF00000704754004D0075
:10F2AC0043004D002D0031003600340030002000AA
:10F2BC0028007600690072007400750061006C0013
:10F2CC00200043004F004D002900200054004D0049
:10F2DC0043004D00310036003400000000000000F7
:10F2EC000000000009024300020100C032090400C2
:10F2FC000001020201000524001001052401000197
:10F30C00042402020524060001070582030800FFFD
:10F31C0009040100020A0000000705030240000076
:10F32C000705810240000000040309042603540071
:10F33C00720069006E0061006D00690063004D0091
:10F34C006F00740069006F006E00200043007400B1
:10F35C006C0000005515AC6A004001C0ABEA579533
:10F36C006B7FD87EB87DA07C8F7B857A82798578FF
:10F37C000878147726763D7559747B73A1723672B2
:10F38C0064719670CC6F076F456EE66D2A6D726C6A
:10F39C00BE6B0D6B5F6AB5696169BB68196879678B
:10F3AC00DC664266AB656065CC643B64AD63206330
:10F3BC0096620F62CB614761C4604460C65F495F6F
:10F3CC00CE5E925E1A5EA45D2F5DBD5C4B5CDC5B19
:10F3DC00A55B385BCC5A625AF95992592C59F95899
:10F3EC0095583358D15771571257B4560000C9006D
:10F3FC0092015B022403ED03B6047F054806110756
:10F40C00D907A2086A09330AFB0AC40B8C0C540DE9
:10F41C001C0EE30EAB0F72103A110112C8128F13AF
:10F42C0055141C15E215A8166E173318F918BE19C9
:10F43C00821A471B0B1CCF1C931D571E1A1FDD1F56
:10F44C009F2061212322E522A62367242825E82575
:10F45C00A82667272628E528A329612A1F2BDC2B41
:10F46C00992C552D112ECC2E872F4130FB30B531D8
:10F47C006E322633DF3396344D350436BA366F3759
:10F48C002438D9388C39403AF23AA53B563C073DE2
:10F49C00B83D683E173FC53F73402141CE417A428B
:10F4AC002543D0437A442445CD4575461C47C34774
:10F4BC0069480F49B449584AFB4A9D4B3F4CE04CB4
:10F4CC00814D204EBF4E5D4FFB4F97503351CE5167
:10F4DC00685202539B533254C9546055F5558A56A1
:10F4EC001D57B0574258D3586459F359825A0F5B81
:10F4FC009C5B285CB35C3E5DC75D4F5ED75E5D5F19
:10F50C00E35F6860EB606E61F0617162F162706381
:10F51C00EE636C64E8646365DD655666CF664667CA
:10F52C00BC673268A66819698B69FD696D6ADC6A0B
:10F53C004A6BB76B236C8E6CF86C616DC96D306E59
:10F54C00966EFB6E5E6FC16F22708370E2704071BD
:10F55C009D71F9715472AE7207735E73B5730A7450
:10F56C005F74B27404755575A575F37541768D7617
:10F57C00D87622776B77B377FA773F788478C77829
:10F58C0009794A798979C879057A417A7C7AB67A87
:10F59C00EE7A267B5C7B917BC57BF87B297C597C46
:10F5AC00887CB67CE37C0E7D397D627D897DB07D67
:10F5BC00D57DFA7D1D7E3E7E5F7E7E7E9C7EB97EF5
:10F5CC00D57EEF7E097F217F377F4D7F617F747FF2
:10F5DC00867F977FA67FB47FC17FCD7FD87FE17F69
:10F5EC00E97FF07FF57FF97FFD7FFE7F0000000053
:10F5FC0010000000160000001B000000200000009E
:10F60C0023000000270000002A0000002D0000004D
:10F61C003000000032000000350000003700000010
:10F62C00390000003B0000003D00000040000000DD
:10F63C0041000000430000004500000047000000AE
:10F64C00490000004B0000004C0000004E00000080
:10F65C005000000051000000530000005400000056
:10F66C005600000057000000590000005A0000002E
:10F67C005B0000005D0000005E0000006000000008
:10F68C0061000000620000006300000065000000E3
:10F69C006600000067000000680000006A000000BF
:10F6AC006B0000006C0000006D0000006E0000009C
:10F6BC007000000071000000720000007300000078
:10F6CC007400000075000000760000007700000058
:10F6DC0078000000790000007A0000007B00000038
:10F6EC007C0000007D0000007E0000008000000017
:10F6FC0080000000810000008200000083000000F8
:10F70C0084000000850000008600000087000000D7
:10F71C0088000000890000008A0000008B000000B7
:10F72C008C0000008D0000008E0000008F00000097
:10F73C00900000009000000091000000920000007A
:10F74C00930000009400000095000000960000005B
:10F75C00960000009700000098000000990000003F
:10F76C009A0000009B0000009B0000009C00000021
:10F77C009D0000009E0000009F000000A000000003
:10F78C00A0000000A1000000A2000000A3000000E7
:10F79C00A3000000A4000000A5000000A6000000CB
:10F7AC00A7000000A7000000A8000000A9000000AE
:10F7BC00AA000000AA000000AB000000AC00000092
:10F7CC00AD000000AD000000AE000000AF00000076
:10F7DC00B0000000B0000000B1000000B20000005A
:10F7EC00B2000000B3000000B4000000B50000003F
:10F7FC00B5000000B6000000B7000000B700000024
:10F80C00B8000000B9000000B9000000BA00000008
:10F81C00BB000000BB000000BC000000BD000000ED
:10F82C00BD000000BE000000BF000000C0000000D2
:10F83C00C0000000C1000000C1000000C2000000B8
:10F84C00C3000000C3000000C4000000C50000009D
:10F85C00C5000000C6000000C7000000C700000083
:10F86C00C8000000C9000000C9000000CA00000068
:10F87C00CB000000CB000000CC000000CC0000004E
:10F88C00CD000000CE000000CE000000CF00000034
:10F89C00D0000000D0000000D1000000D10000001A
:10F8AC00D2000000D3000000D3000000D400000000
:10F8BC00D4000000D5000000D6000000D6000000E7
:10F8CC00D7000000D7000000D8000000D9000000CD
:10F8DC00D9000000DA000000DA000000DB000000B4
:10F8EC00DB000000DC000000DD000000DD0000009B
:10F8FC00DE000000DE000000DF000000E000000081
:10F90C00E0000000E1000000E1000000E200000067
:10F91C00E2000000E3000000E3000000E40000004F
:10F92C00E5000000E5000000E6000000E600000035
:10F93C00E7000000E7000000E8000000E80000001D
:10F94C00E9000000EA000000EA000000EB00000003
:10F95C00EB000000EC000000EC000000ED000000EB
:10F96C00ED000000EE000000EE000000EF000000D3
:10F97C00F0000000F0000000F1000000F1000000B9
:10F98C00F2000000F2000000F3000000F3000000A1
:10F99C00F4000000F4000000F5000000F500000089
:10F9AC00F6000000F6000000F7000000F700000071
:10F9BC00F8000000F8000000F9000000F900000059
:10F9CC00FA000000FA000000FB000000FB00000041
:10F9DC00FC000000FC000000FD000000FD00000029
:10F9EC00FE000000FE000000FF0000000000000010
:10F9FC0001020304010203040607080902040608B5
:10FA0C000200000000000001313634305632303232
:04FA1C0000000000E6
:10FA2000AC00000040000000FB070000FF070000E2
:10FA3000000800000500000014FA00080B0C0D0A75
:10FA40000E08090001000000020000000300000091
:10FA5000040000000000004001000000000400401D
:10FA60000101010100C201000000080034F3000898
:10FA70000400000038F3000826000000C000002049
:10FA800032000000F40000201A000000F0F200082C
:10FA900043000000AC000020120000004588000870
:10FAA0004986000895840008A9840008AD840008F0
:10FAB0000D85000831850008398600082986000870
:10FAC000058600080000000040000000120110013F
:10FAD00002000040D01600000202010203010000F3
:10FAE000320354004D0043004D002D003000300023
:10FAF0003000300020002800760069007200740099
:10FB0000750061006C00200043004F004D0029008B
:10FB1000200000001A0354004D0043004D00300047
:10FB20003000300030000000000000000000000045
:10FB30009583000815BC000815BC000815BC00081A
:10FB400015BC000815BC000815BC000815BC000851
:10FB500015BC00089987000815BC000815BC0008F2
:10FB600015BC000815BC00080401000015BC000805
:10FB70007184000815BC000815BC000815BC0008FD
:10FB800015BC000815BC000815BC000889840008D5
:08FB900001000000010000006B
:040000050800410CA2
:00000001FF
